:100000000C94BB010C94FA310C9427320C94E3014C
:100010000C94E3010C94E3010C94E3010C94E301D0
:100020000C94E3010C94E3010C94E3010C94CE06D0
:100030000C94E3010C94E3010C94E3010C94E301B0
:100040000C9406310C94E3010C9444060C94800645
:100050000C94E3010C94E3010C94E3010C94E30190
:100060000C94E3010C94E301084AD73B3BCE016EAC
:1000700084BCBFFDC12F3D6C74319ABD56833DDAFF
:100080003D00C77F11BED9E4BB4C3E916BAAAABE0E
:10009000000000803F05A84CCDB2D44EB93836A937
:1000A000020C50B9918688083CA6AAAA2ABE000074
:1000B00000803F0664EC1B3C04BC163E3BE5B93CAB
:1000C000C93C37C29E5A3D660498083EEA69AAAA0E
:1000D0003E000000803F2020BF0020BF00BF007C0A
:1000E0002020202020202020202020202020202010
:1000F00020202000C8202020202020202020202078
:1001000020C900C8202020202020202020202020BE
:10011000C97C00D820202020202020202020202042
:10012000D97C00C820202020202020202020202032
:10013000C97C00C820202020202020202020202032
:10014000C97C00207265766F00206172737369004C
:100150006D696E6F706F7364206C6962726570692F
:100160006C6F74002020202020BABBBCBDBE7C2058
:1001700020202020CACBCCCDCE7C00626F6F74696A
:100180006E672075703AEDF2F2F2F2F2F2F2F300DD
:1001900062617474657279207761726E696E67202E
:1001A0000074787069642076616C756573006261B3
:1001B000726F2074656D700074656D706469737022
:1001C00020006163746976652000706173736976DD
:1001D000650075617674616C6B2000736574757071
:1001E0002073637265656E7C7C7C0043686172205D
:1001F000446F6E650A00526561647920666F7220F3
:10020000466F6E740A0055706461746520436861BE
:10021000725365740000407A10F35A00A0724E18B1
:10022000090010A5D4E80000E87648170000E40BA8
:1002300054020000CA9A3B000000E1F5050000806E
:10024000969800000040420F000000A086010000C8
:1002500000102700000000E8030000000064000018
:100260000000000A00000000000100000000002C57
:1002700076D888DC674F0823DFC1DFAE59E1B1B71C
:1002800096E5E3E453C63AE651997696E8E6C284E9
:1002900026EB898C9B62ED407C6FFCEFBC9C9F4001
:1002A000F2BAA56FA5F490055A2AF75C936B6CF926
:1002B000676DC11BFCE0E40D47FEF520E6B500D0FC
:1002C000ED902E0300943577050080841E08000011
:1002D000204E0A000000C80C333333330F986E12DF
:1002E000831141EF8D2114893BE65516CFFEE6DBE5
:1002F00018D1844B381BF77C1D901DA4BBE424202F
:100300003284725E228100C9F124ECA1E53D276EA2
:10031000616E00696E660000000000240027002A5C
:100320000000000000250028002B00000000002332
:100330000026002900040404040404040402020248
:100340000202020303030303030102040810204016
:10035000800102040810200102040810200000009F
:100360000700020100000304060000000000000076
:1003700000004F04150811241FBECFEFD8E0DEBFE8
:10038000CDBF13E0A0E0B1E0E6EEFEE602C00590CE
:100390000D92A83DB107D9F716E0A8EDB3E001C072
:1003A0001D92AA38B107E1F713E0C6E7D3E004C015
:1003B0002297FE010E946D37C237D107C9F70E940C
:1003C00036330C9471370C940000FA01AA272830B8
:1003D00051F1203181F1E8946F936E7F6E5F7F4F12
:1003E0008F4F9F4FAF4FB1E03ED0B4E03CD0670F8E
:1003F000781F891F9A1FA11D680F791F8A1F911DE1
:10040000A11D6A0F711D811D911DA11D20D009F430
:1004100068943F912AE0269F11243019305D319372
:10042000DEF6CF010895462F4770405D4193B3E05B
:100430000FD0C9F7F6CF462F4F70405D4A3318F002
:10044000495D31FD4052419302D0A9F7EACFB4E0B3
:10045000A6959795879577956795BA95C9F700976B
:100460006105710508959B01AC010A2E069457950C
:10047000479537952795BA95C9F7620F731F841F63
:10048000951FA01D0895283008F027E03327DA01D2
:10049000990F311D87FD916000966105710539F452
:1004A00032602E5F3D9330E32A95E1F708959F3F38
:1004B00030F080387105610509F03C5F3C5F3D9389
:1004C000913008F08068911DDF93CF931F930F93B5
:1004D000FF92EF92192F987F9695E92F9695969512
:1004E000E90FFF27E159FD4F99273327EE24FF2419
:1004F000A701E70105900894079428F4360FE71E3A
:10050000F81E491F511D660F771F881F991F0694FB
:10051000A1F70590079428F4E70EF81E491F561F0F
:10052000C11D770F881F991F661F0694A1F70590BC
:10053000079428F4F80E491F561FC71FD11D880FB6
:10054000991F661F771F0694A1F70590079420F462
:10055000490F561FC71FD81F990F661F771F881F87
:100560000694A9F784911095177041F0D695C79518
:1005700057954795F794E7941A95C1F7E5E1F2E0AE
:1005800068941590159135916591959105907FE24C
:100590007395E118F10A430B560BC90BD009C0F74C
:1005A000E10CF11E431F561FC91FD01D7EF470338E
:1005B00011F48A95E6CFE894015030F0080F0AF460
:1005C0000027021708F4202F2395022F7A3328F0F2
:1005D00079E37D932A95E9F710C07D932A9589F6F2
:1005E000069497956795379517951794E118F10A32
:1005F000430B560BC90BD00998F023957E91739548
:100600007A3308F070E37C932013B8F77E91706121
:100610007D9330F0839571E37D9370E32A95E1F744
:100620001124EF90FF900F911F91CF91DF919927A7
:1006300087FD90950895CF93DF93BC01823091059B
:1006400010F462E070E0A0918806B0918906ED0197
:1006500040E050E0E0E0F0E021C088819981861719
:10066000970769F48A819B81309719F0938382837D
:1006700004C09093890680938806FE0134C06817F1
:10068000790738F44115510519F08417950708F4D6
:10069000AC01FE018A819B819C01E9012097E9F66A
:1006A00041155105A9F1CA01861B970B049708F45F
:1006B000BA01E0E0F0E02AC08D919C911197841777
:1006C0009507F9F46417750781F412968D919C9142
:1006D0001397309719F09383828304C0909389060F
:1006E00080938806FD0132964CC0CA01861B970B89
:1006F000FD01E80FF91F6193719302978D939C930D
:1007000040C0FD01828193819C01D9011097A1F61F
:100710008091860690918706892B41F48091790219
:1007200090917A02909387068093860640917B028F
:1007300050917C024115510541F44DB75EB780914F
:10074000770290917802481B590B209186063091D0
:100750008706CA01821B930B8617970780F0AB01AF
:100760004E5F5F4F8417950750F0420F531F509311
:10077000870640938606F9016193719302C0E0E019
:10078000F0E0CF01DF91CF910895CF93DF930097F1
:1007900009F450C0EC0122971B821A82A0918806AE
:1007A000B0918906109709F140E050E0AC17BD0701
:1007B00008F1BB83AA83FE0121913191E20FF31F5F
:1007C000AE17BF0779F48D919C911197280F391FAF
:1007D0002E5F3F4F3983288312968D919C911397FA
:1007E0009B838A834115510571F4D0938906C09388
:1007F000880620C012968D919C911397AD010097A9
:1008000011F0DC01D3CFFA01D383C283219131915E
:10081000E20FF31FCE17DF0769F488819981280F53
:10082000391F2E5F3F4FFA01318320838A819B81DC
:1008300093838283DF91CF910895FC0105906150ED
:1008400070400110D8F7809590958E0F9F1F0895E6
:10085000FC016150704001900110D8F7809590958F
:100860008E0F9F1F08956EBD0DB407FEFDCF8EB590
:1008700008958DE061E00E9454328BE061E00E94B7
:1008800054328CE060E00E9454328AE061E00E94C1
:1008900054321CBC80E58CBD8DB58EB5089588EDB5
:1008A00093E00E9439040895FC011382128288EEBD
:1008B00093E0A0E0B0E084839583A683B7838EE8BD
:1008C00092E0918380830895FC018089803419F43B
:1008D00021E030E002C020E030E0C9010895FC01D1
:1008E000818990E00895FC01648745876687478782
:1008F000089580E090E0089580E090E0089580E021
:1009000090E008950895EF92FF921F93CF93DF93A5
:10091000162F7A0186E060E00E94933288ED93E022
:1009200060E00E94330488ED93E060E00E943304AD
:1009300088ED93E069E00E94330488ED93E0612F35
:100940000E943304C0E0D0E0F701EC0FFD1F1081DE
:1009500088ED93E06AE00E94330488ED93E06C2F09
:100960000E94330488ED93E06BE00E94330488ED2D
:1009700093E0612F0E9433042196C633D10521F7FD
:1009800088ED93E068E00E94330488ED93E060EA2C
:100990000E94330488ED93E060EA0E94330485FDF1
:1009A000F9CF88ED93E060E00E94330488ED93E096
:1009B0006CE00E94330486E061E00E949332DF9194
:1009C000CF911F91FF90EF9008951F93CF93DF93E6
:1009D000EC01162F86E060E00E94933288ED93E0F0
:1009E00060E00E943304112319F0113059F404C05F
:1009F00088ED93E0688904C068896C6188ED93E0B4
:100A00000E94330486E061E00E949332DF91CF912F
:100A10001F910895EF92FF920F931F938EE1489FCD
:100A200070011124E60EF11C86E060E00E94933212
:100A300008ED13E0C80165E00E943304C8016F2D82
:100A40000E943304C80166E00E943304C8016E2D81
:100A50000E9433041F910F91FF90EF900895EF9241
:100A6000FF920F931F937C0108ED13E0C80167E02C
:100A70000E943304C8016FEF0E94330486E061E0F6
:100A80000E949332F70187858F5F87871F910F91AF
:100A9000FF90EF900895EF92FF920F931F93FC0148
:100AA000E7848EE1E89E700111248685E80EF11C32
:100AB00086E060E00E94933208ED13E0C80164E034
:100AC0000E943304C80163E00E943304C80165E05A
:100AD0000E943304C8016F2D0E943304C80166E0F0
:100AE0000E943304C8016E2D0E9433041F910F91A0
:100AF000FF90EF9008951F93CF93DF93EC01162F93
:100B00006C3731F40E942F05CE010E944B050AC0BC
:100B100088ED93E067E00E94330488ED93E0612F55
:100B20000E94330481E090E0DF91CF911F910895FE
:100B30000F931F9386E060E00E94933208ED13E06C
:100B4000C80164E00E943304C80164E00E943304D9
:100B500086E061E00E9493321F910F9108951F93E8
:100B6000CF93DF93EC01188A16E0198B86E796E0A5
:100B700060E973E00E946630813049F480E4888B3C
:100B800088E0898B86E060E00E94933202C0188A78
:100B9000198B86E060E00E949332DF91CF911F9124
:100BA00008950F931F93CF93DF93EC0186E061E0EC
:100BB0000E94543282E060E00E94543282E061E0A0
:100BC0000E949332CE010E94AF0586E060E00E9451
:100BD000933288ED93E06CEE0E94330488ED93E04D
:100BE0006FEF0E943304182F88ED93E060E00E94BD
:100BF00033046889626088ED93E00E94330462E305
:100C000070E080E090E00E945C3188ED93E06CE65B
:100C10000E9433041F7E88ED93E0612F0E9433040D
:100C20008889803419F00DE010E002C000E110E086
:100C30001092DA031092D90317C06091D903709112
:100C4000DA03605F88ED93E00E94330488ED93E05F
:100C500069E00E9433048091D9039091DA030196F0
:100C60009093DA038093D9038091D9039091DA03AA
:100C70008017910714F3CE0161E00E94E504DF9133
:100C8000CF911F910F9108951F920F920FB60F925F
:100C900011242F933F934F938F939F93EF93FF9341
:100CA0004091C60020916506309166062F5F3F4F48
:100CB0008091690690916A062823392380916706FE
:100CC000909168062817390779F080916506909110
:100CD0006606E0916B06F0916C06E80FF91F408301
:100CE0003093660620936506FF91EF919F918F9157
:100CF0004F913F912F910F900FBE0F901F9018951D
:100D00001F920F920FB60F9211242F933F938F9340
:100D10009F93EF93FF9320916F063091700680911F
:100D20006D0690916E0628173907E9F080916F06DD
:100D300090917006E0917306F0917406E80FF91F28
:100D400080818093C60080916F0690917006019615
:100D5000209171063091720682239323909370063E
:100D600080936F0610C020916D0630916E068091C1
:100D70006F06909170062817390729F48091C100F9
:100D80008F7D8093C100FF91EF919F918F913F9153
:100D90002F910F900FBE0F901F9018951F920F92DA
:100DA0000FB60F9211248F939F9380919B04909183
:100DB0009C04892B51F080919D0490919E04019692
:100DC00090939E0480939D0409C080919F0490910C
:100DD000A00401969093A00480939F049F918F910B
:100DE0000F900FBE0F901F901895CF93DF93482F51
:100DF000EB018091FB05833009F45DC0843028F459
:100E00008130C1F0823058F50AC0853009F4D2C073
:100E1000853008F4A8C0863009F0F2C0E9C04C3330
:100E200009F0EEC081E08093FB05488384EB80935A
:100E3000FA05E6C0842F90E0E091FA05F0E0E8279B
:100E4000F927E456FD4F20812093FA05887F9070A2
:100E5000809741F582E08093FB05498329C0242FC8
:100E600030E0E091FA05F0E0E227F327E456FD4F89
:100E700080818093FA058091F9058F5F8093F90551
:100E8000823018F43B832A83BBC0922F88272A81A3
:100E90003B81820F931F9B838A830A978F3F910523
:100EA00021F018F01092FB05ABC083E08093FB05A6
:100EB0001092F905A5C0E42FF0E08091FA0590E0CA
:100EC000E827F927E456FD4F80818093FA05609169
:100ED000F9056F5F6093F905623089F0633020F4A3
:100EE000613009F08DC006C0633091F0643009F0C4
:100EF00087C022C0842F90E0A0E0B0E018C0242F6B
:100F000030E040E050E0542F432F322F222707C01B
:100F1000242F30E040E050E0A901332722278C81C4
:100F20009D81AE81BF81820F931FA41FB51F8C834B
:100F30009D83AE83BF8364C0242F30E040E050E047
:100F4000522F4427332722278C819D81AE81BF8178
:100F5000820F931FA41FB51F8C839D83AE83BF8315
:100F60006093FB05A5CF242F30E0E091FA05F0E077
:100F7000E227F327E456FD4F80818093FA058091A4
:100F8000F9058F5F8093F905813019F08230C1F542
:100F900003C03987288734C0922F88272885398550
:100FA000280F391F398728878A819B810A97F1F09A
:100FB00085E07CCFE42FF0E08091FA0590E0E8270F
:100FC000F927E456FD4F80818093FA052091F905B9
:100FD0002F5F2093F90530E0FB01E20FF31F4187FB
:100FE0008A819B810A972817390750F086E05ECFE7
:100FF000C75FDE4F4883C950D14087E08093FB052F
:101000008091FB05873069F41092FB05C75FDE4FC6
:101010009091FA058881C950D140981711F48A81BE
:1010200001C080E0DF91CF9108958F92AF92CF926F
:10103000EF92FF920F931F9381E694E060E045ECFE
:1010400050E024EC30E000EC10E0B1ECEB2EF12CA1
:10105000CC24C394A8E9AA2EF0E28F2E0E94D629B0
:101060008EE794E00E94540410929104109292042E
:101070001092930410929404109295041092960486
:10108000109297041092980410929A041092990466
:10109000109290041F910F91FF90EF90CF90AF901E
:1010A0008F900895AF92BF92CF92DF92EF92FF920E
:1010B0000F931F93E0906106F09062060091630623
:1010C000109164068FE590E0A0E0B0E0E80EF91E14
:1010D0000A1F1B1F0E944E316E157F058007910766
:1010E00008F44EC0A090C604B090C704C090C804D5
:1010F000D090C904C601B50120E030E040E85FE3CC
:101100000E94D635181694F5E0901906F0901A064C
:1011100000911B0610911C060E944E312091610621
:10112000309162064091630650916406621B730B16
:10113000840B950B0E94AC349B01AC01C601B50138
:101140000E94E13520E030E04AE754E40E94133485
:101150009B01AC01C801B7010E9446336093190698
:1011600070931A0680931B0690931C060E944E31C2
:1011700060936106709362068093630690936406A1
:101180001F910F91FF90EF90DF90CF90BF90AF90A5
:101190000895DF93CF9300D000D0CDB7DEB7FB0129
:1011A000E80FF91F628583859485258569838A8385
:1011B0009B832C83492F5C81782FCA010F900F905D
:1011C0000F900F90CF91DF910895AF92BF92DF9271
:1011D000EF92FF920F931F93CF93DF938C01809137
:1011E000FC0580FDE4C0F801F08081E694E06F2DFD
:1011F0000E94B72AE801C75FDE4FEF2DF0E0E4560A
:10120000FD4F80818883F801F18081E694E06F2DA5
:101210000E94B72AEF2DF0E0888190E0E827F927B7
:10122000E456FD4F80818883F801F28081E694E0E6
:101230006F2D0E94B72AEF2DF0E0888190E0E8271B
:10124000F927E456FD4F80818883F801F38081E619
:1012500094E06F2D0E94B72AEF2DF0E0888190E096
:10126000E827F927E456FD4F80818883F801F48050
:1012700081E694E06F2D0E94B72AEF2DF0E088817F
:1012800090E0E827F927E456FD4F80818883F80134
:101290002481358146815781232F342F452F5527AF
:1012A000F22E81E694E0622F0E94B72AEF2DF0E043
:1012B000888190E0E827F927E456FD4F80818883F4
:1012C000F80124813581468157819A0144275527A9
:1012D000F22E81E694E0622F0E94B72AEF2DF0E013
:1012E000888190E0E827F927E456FD4F80818883C4
:1012F000F8012481358146815781252F33274427E2
:101300005527F22E81E694E0622F0E94B72AEF2D36
:10131000F0E0888190E0E827F927E456FD4F8081CE
:10132000888381E694E060E00E94B72AE881F0E0DB
:10133000E456FD4F8081888381E694E060E00E945E
:10134000B72AE881F0E0E456FD4F80818883F801F8
:10135000828193810B9718F18AE0A82EB12CA00E00
:10136000B11E750112C0F701D1907F0181E694E0B2
:101370006D2D0E94B72AED2DF0E0888190E0E827DE
:10138000F927E456FD4F808188832E2D2A1930E0FD
:10139000F801828193810A972817390720F3075FA4
:1013A0001E4F81E694E0F80160810E94B72ADF9128
:1013B000CF911F910F91FF90EF90DF90BF90AF9072
:1013C0000895DF93CF93CDB7DEB7CA50D1400FB6A3
:1013D000F894DEBF0FBECDBF2CE329836A832AE0D9
:1013E00030E03C832B83FC0184819581A681B78109
:1013F0008D839E83AF83B887CE0101960E94E50856
:10140000C65FDE4F0FB6F894DEBF0FBECDBFCF91E3
:10141000DF91089586E796E06AE773E00E94663000
:10142000882331F586E696E6A6E6B0E48093FE05CD
:101430009093FF05A0930006B093010680E090E032
:10144000A0E8BFE38093020690930306A0930406EE
:10145000B093050688EE93E0909307068093060606
:1014600081E8809308068DE8809309068DEF25C0FA
:1014700082E598EBAEE0B0E48093FE059093FF0523
:10148000A0930006B093010685E89BEEA1E5B0E4C9
:101490008093020690930306A0930406B09305067A
:1014A00080EA94E190930706809306068BEF809381
:1014B000080686E6809309068AEF80930A06089557
:1014C000FF920F931F9306E716E0C8016CE773E0E5
:1014D0000E94663080934506C8016EE773E00E9463
:1014E000663080934606C80160E873E00E9466306B
:1014F00080932506C8016EE873E00E9466308093F1
:101500003D06C8016AE873E00E94663080933B069E
:10151000C80164E873E00E94663080934706C80102
:1015200066E873E00E94663080934806C8016CE864
:1015300073E00E94663080932D06C80162E973E073
:101540000E94663080934906C80164E973E00E94F6
:10155000663080932C06C80164EF73E00E94663009
:10156000F82EC80165EF73E00E946630382F20E046
:101570002F0D311D30934B0620934A06C80166EFAC
:1015800073E00E946630F82EC80167EF73E00E9496
:101590006630382F20E02F0D311D30934D062093FB
:1015A0004C06C80168EF73E00E946630F82EC8014F
:1015B00069EF73E00E946630382F20E02F0D311D57
:1015C00030934F0620934E06C8016BEF73E00E94E4
:1015D0006630809324061F910F91FF900895BC01FF
:1015E00086E796E00E94663008956091B00470919D
:1015F000B1048091B2049091B30420E030E040E166
:1016000052E40E94E13520E030E044EB53E40E94D4
:1016100013340E9444360E947B349B012550304095
:1016200037FF03C09B01215E3F4FADE0B6E0F901FB
:10163000E456FC4F80818C932F5F3F4F243231055D
:1016400014F020E030E0119686E0A831B80779F771
:101650001C9208952F923F924F925F926F927F92C9
:101660008F929F92AF92BF92CF92DF92EF92FF92B2
:101670000F931F93DF93CF9300D000D000D0CDB74E
:10168000DEB7182F662E2091A6043091A7042A35C4
:10169000310530F0C9018D549F4F89359105E8F42B
:1016A00037FF02C02D543F4FC90137FF03C090954B
:1016B00081959F4F8A3191053CF0F4E48F2E912C57
:1016C000E9ED2E2E312C1DC00A975CF17BE3872EAD
:1016D000912C62ED262E312C20C02B35310514F0D3
:1016E000235B3040C90137FF03C0909581959F4F20
:1016F0008A31910554F056E5852E912C4CED242E1F
:10170000312C37E0A32EB12C15C00A9754F02DE4EC
:10171000822E912C94ED292E312C88E0A82EB12C0C
:1017200009C005E0802E912CB8E32B2E312CA9E0C6
:10173000AA2EB12C6091A8047091A904882777FD86
:101740008095982F0E94AE3427EA32E94BE25CEB99
:101750000E94E1350E94B53620E030E040EA50E4D6
:101760000E94E13520E030E040E951E40E94E1359B
:101770000E94443620E030E044E352E40E944633C5
:101780000E947B34712EFEEBCF2EFFEFDF2E9B01EC
:10179000442737FD4095542F29833A834B835C833C
:1017A000EEE74E2EE4E05E2E4AEF5FEF240E351E8C
:1017B0006091A6047091A704882777FD8095982FE3
:1017C0000E94AE3425E33AEF4EE85CE30E94E13537
:1017D0000E94B5367B018C01B601882777FD809584
:1017E000982F0E94AE349B01AC01C801B7010E9442
:1017F000E1357B018C0169817A818B819C810E941A
:10180000AE349B01AC01C801B7010E9446330E946F
:101810007B349B01CB0101978A35910508F071C09B
:1018200062E170E00E941B378B012F5F3F4FAEEEED
:10183000BFEF6A9FC0016B9F900D7A9F900D11249E
:10184000820F931F62E070E00E941B376D837E83DE
:10185000E62CE01A4E2D4C5F8EE794E0672D0E9437
:101860000A0500D000D000D0EDB7FEB73196ADB775
:10187000BEB712965C924E92119720E031E033830E
:1018800022838D819E81880D991D958384830E947A
:10189000B5294DB75EB74A5F5F4F0FB6F8945EBF8C
:1018A0000FBE4DBF8D819E818A159B0554F104307A
:1018B00011053CF593E0E90EC201672D4E2D0E9403
:1018C0000A0500D000D000D0EDB7FEB73196ADB715
:1018D000BEB712965C924E92119720E031E03383AE
:1018E00022834D815E81420D531D558344830E94A6
:1018F000B5298DB79EB706960FB6F8949EBF0FBE5A
:101900008DBFACE0B0E0CA0EDB1E7394BEE4CB1614
:10191000D10409F04DCF26960FB6F894DEBF0FBE66
:10192000CDBFCF91DF911F910F91FF90EF90DF908E
:10193000CF90BF90AF909F908F907F906F905F906F
:101940004F903F902F900895823010F422E002C013
:10195000282F220F30E08DB79EB708970FB6F89466
:101960009EBF0FBE8DBFEDB7FEB731968EE794E0F8
:10197000ADB7BEB712969C938E93119783E091E01A
:101980009383828322573F4F358324832F5F3F4FBA
:10199000378326830E94B5298DB79EB708960FB668
:1019A000F8949EBF0FBE8DBF0895CF93DF93AC0117
:1019B000E091B804F091B90420910B0630910C0627
:1019C000C9018C599F4F8E179F071CF4EA0121977C
:1019D00009C024563040E217F30714F0EA0102C0B0
:1019E000EA012196842F90E0C817D90729F086E7ED
:1019F00096E04C2F0E946D30CE01DF91CF9108957B
:101A00000F931F9306E716E0C80163EF73E041E010
:101A10000E946D30C80164EF73E043E10E946D30B5
:101A2000C80165EF73E046E00E946D30C80166EFC3
:101A300073E040E10E946D30C80167EF73E047E258
:101A40000E946D30C80168EF73E048E80E946D3075
:101A5000C80169EF73E043E10E946D301F910F915F
:101A60000895CF92DF92EF92FF920F931F937C0124
:101A7000D62EC72E0EE714E0C8016E2D4D2D0E9404
:101A80007304C8010E944B0500D000D0EDB7FEB72B
:101A90001283018383E391E0948383830E94A429CA
:101AA000EDB7FEB71283018383E291E094838383D1
:101AB0000E94A429EDB7FEB71283018383E191E070
:101AC000948383830E94A429EDB7FEB71283018318
:101AD00083E091E0948383830E94A429EDB7FEB74D
:101AE0001283018384EF90E0948383830E94A4296E
:101AF0000F900F900F900F90C8010E942F05C70103
:101B000001966D2D7C2D0E942A0B1F910F91FF9045
:101B1000EF90DF90CF900895AF92BF92CF92DF9277
:101B2000EF92FF920F931F93B82EA62E0E944E3174
:101B300028EE33E040E050E00E942E3779018A0120
:101B4000AEE7CA2EA4E0DA2EC6016B2D4A2D0E9404
:101B50007304C6010E944B05A090D604B090D70430
:101B60008DB79EB744970FB6F8949EBF0FBE8DBF3A
:101B7000EDB7FEB73196ADB7BEB71296DC92CE92F6
:101B8000119788E091E09383828383EB90E09583C3
:101B90008483C7016CE370E00E941B37CB016CE3C8
:101BA00070E00E941B37978386832AE330E03187F9
:101BB0002087C7016CE370E00E941B379387828700
:101BC00085E690E095878487C5016CE370E00E940C
:101BD0000737CB016CE370E00E941B37978786873D
:101BE000318B208BC5016CE370E00E940737938B2B
:101BF000828B0E94B5298DB79EB744960FB6F89494
:101C00009EBF0FBE8DBFC6010E942F051F910F9171
:101C1000FF90EF90DF90CF90BF90AF900895EF923C
:101C2000FF920F931F93282F462FBEE7EB2EB4E0B1
:101C3000FB2EC701622F0E947304C7010E944B054F
:101C40008DB79EB70A970FB6F8949EBF0FBE8DBF93
:101C50000DB71EB70F5F1F4FEDB7FEB7F282E182DF
:101C600080E291E0F801938382836091D8047091BF
:101C7000D9048091DA049091DB042091020630911E
:101C8000030640910406509105060E94E135F801D3
:101C9000648375838683978380EB90E09187808748
:101CA0000E94B5298DB79EB70A960FB6F8949EBFCD
:101CB0000FBE8DBFC7010E942F051F910F91FF908E
:101CC000EF9008958F929F92AF92BF92CF92DF9242
:101CD000EF92FF920F931F93E82EF62E0EE714E07B
:101CE000C8016E2D4F2D0E947304C8010E944B0540
:101CF0008DB79EB70C970FB6F8949EBF0FBE8DBFE1
:101D0000EDB7FEB73196ADB7BEB712961C930E93E2
:101D1000119728E2822E21E0922E938282829DEEFC
:101D2000A92EB12CB582A4828091E1049091E204A5
:101D3000A091E304B091E40486839783A087B187E0
:101D400083EFC82ED12CD386C2860E94B5298DB7C9
:101D50009EB70C960FB6F8949EBF0FBE8DBFC801FC
:101D60000E942F05F394C8016E2D4F2D0E9473041D
:101D7000C8010E944B05ADB7BEB71C970FB6F894CB
:101D8000BEBF0FBEADBFEDB7FEB7319612961C9326
:101D90000E93119793828282B582A4828091E5048A
:101DA0009091E604A091E704B091E80486839783BC
:101DB000A087B187D386C2860E94B5298DB79EB70A
:101DC0000C960FB6F8949EBF0FBE8DBFC8010E943F
:101DD0002F05F394C8016E2D4F2D0E947304C80186
:101DE0000E944B05ADB7BEB71C970FB6F894BEBFA7
:101DF0000FBEADBFEDB7FEB7319612961C930E9392
:101E0000119793828282B582A4828091E904909195
:101E1000EA04A091EB04B091EC0486839783A08739
:101E2000B187D386C2860E94B5298DB79EB70C961E
:101E30000FB6F8949EBF0FBE8DBFC8010E942F053C
:101E40001F910F91FF90EF90DF90CF90BF90AF90D8
:101E50009F908F9008950F931F93282F462F0EE782
:101E600014E0C801622F0E947304C8010E944B0550
:101E70008DB79EB70A970FB6F8949EBF0FBE8DBF61
:101E8000EDB7FEB73196ADB7BEB712961C930E9361
:101E9000119782E391E09383828389EB90E09583AD
:101EA00084838091D4049091D5049783868382E8BB
:101EB00090E0918780870E94B5298DB79EB70A96DA
:101EC0000FB6F8949EBF0FBE8DBFC8010E942F05AC
:101ED0001F910F910895EF92FF920F931F93282F58
:101EE000462F3EE7E32E34E0F32EC701622F0E9417
:101EF0007304C7010E944B058DB79EB70C970FB6B0
:101F0000F8949EBF0FBE8DBF0DB71EB70F5F1F4F5A
:101F1000EDB7FEB7F282E1828AE391E0F8019383A4
:101F2000828384EE90E0958384836091D2047091E3
:101F3000D304882777FD8095982F0E94AE342AE03D
:101F400037ED43E25CE30E94E135F8016683778375
:101F5000808791878FE890E0938782870E94B529D8
:101F60008DB79EB70C960FB6F8949EBF0FBE8DBF6F
:101F7000C7010E942F051F910F91FF90EF900895C8
:101F80000F931F93282F462F0EE714E0C801622FEE
:101F90000E947304C8010E944B058DB79EB70C9731
:101FA0000FB6F8949EBF0FBE8DBFEDB7FEB731964A
:101FB000ADB7BEB712961C930E9311978AE391E0CA
:101FC0009383828382EE90E0958384838091CE0414
:101FD0009091CF04A091D004B091D10486839783CF
:101FE000A087B1878EE890E0938782870E94B52909
:101FF0008DB79EB70C960FB6F8949EBF0FBE8DBFDF
:10200000C8010E942F051F910F9108950F931F93F0
:10201000282F462F8EE794E0622F0E9473048EE7EC
:1020200094E00E944B058091B504882319F424E4C0
:1020300031E057C0813019F428E431E052C08230D9
:1020400019F42CE431E04DC0833019F420E531E07F
:1020500048C0843019F424E531E043C0853019F4D8
:1020600028E531E03EC0863019F42CE531E039C076
:10207000873019F420E631E034C0883019F424E6C2
:1020800031E02FC0893019F428E631E02AC08A30C7
:1020900019F42CE631E025C08B3019F420E731E04B
:1020A00020C08C3019F424E731E01BC08D3019F4C6
:1020B00028E731E016C08E3019F42CE731E011C06A
:1020C0008F3019F420E831E00CC0803119F424E895
:1020D00031E007C0813119F028E831E002C029E879
:1020E00031E08DB79EB708970FB6F8949EBF0FBE2C
:1020F0008DBFEDB7FEB731960EE714E0ADB7BEB7B2
:1021000012961C930E9311978DE891E0938382832E
:1021100080EE90E095838483378326830E94B529DF
:102120008DB79EB708960FB6F8949EBF0FBE8DBFB1
:10213000C8010E942F051F910F9108950F931F93BF
:10214000282F462F0EE714E0C801622F0E94730467
:10215000C8010E944B058DB79EB70A970FB6F89439
:102160009EBF0FBE8DBFEDB7FEB73196ADB7BEB700
:1021700012961C930E93119782E991E093838283C8
:1021800087E890E0958384838091B6049091B704AA
:102190009783868385E290E0918780870E94B529A6
:1021A0008DB79EB70A960FB6F8949EBF0FBE8DBF2F
:1021B000C8010E942F051F910F9108950F931F933F
:1021C000282F462F0EE714E0C801622F0E947304E7
:1021D000C8010E944B058DB79EB70A970FB6F894B9
:1021E0009EBF0FBE8DBFEDB7FEB73196ADB7BEB780
:1021F00012961C930E9311978CE991E0938382833E
:102200008091A8049091A9049583848380EB90E049
:102210009783868381EB90E0918780870E94B52920
:102220008DB79EB70A960FB6F8949EBF0FBE8DBFAE
:10223000C8010E942F051F910F9108950F931F93BE
:10224000282F462F0EE714E0C801622F0E94730466
:10225000C8010E944B058DB79EB70A970FB6F89438
:102260009EBF0FBE8DBFEDB7FEB73196ADB7BEB7FF
:1022700012961C930E9311978CE991E093838283BD
:102280008091A6049091A7049583848380EB90E0CD
:102290009783868382EB90E0918780870E94B5299F
:1022A0008DB79EB70A960FB6F8949EBF0FBE8DBF2E
:1022B000C8010E942F051F910F9108950F931F933E
:1022C000282F462F0EE714E0C801622F0E947304E6
:1022D000C8010E944B058DB79EB70A970FB6F894B8
:1022E0009EBF0FBE8DBFEDB7FEB73196ADB7BEB77F
:1022F00012961C930E93119784EA91E09383828344
:1023000081EE90E09583848380918502909186028E
:102310009783868385E290E0918780870E94B52924
:102320008DB79EB70A960FB6F8949EBF0FBE8DBFAD
:10233000C8010E942F051F910F9108950F931F93BD
:10234000282F462F0EE714E0C801622F0E94730465
:10235000C8010E944B058DB79EB70C970FB6F89435
:102360009EBF0FBE8DBFEDB7FEB73196ADB7BEB7FE
:1023700012961C930E9311978CEA91E093838283BB
:1023800086EB91E09583848380ED90E0978386834C
:102390008DE096E09187808781ED90E0938782873A
:1023A0000E94B5298DB79EB70C960FB6F8949EBFC4
:1023B0000FBE8DBFC8010E942F051F910F91089578
:1023C0000F931F93282F462F0EE714E0C801622FAA
:1023D0000E947304C8010E944B058DB79EB70A97EF
:1023E0000FB6F8949EBF0FBE8DBFEDB7FEB7319606
:1023F000ADB7BEB712961C930E93119784EC91E083
:10240000938382838091B0049091B104A091B2042F
:10241000B091B30484839583A683B78380EB90E067
:10242000918780870E94B5298DB79EB70A960FB60F
:10243000F8949EBF0FBE8DBFC8010E942F051F914B
:102440000F9108950F931F93282F462F0EE714E046
:10245000C801622F0E947304C8010E944B058DB70A
:102460009EB70C970FB6F8949EBF0FBE8DBFEDB709
:10247000FEB73196ADB7BEB712961C930E93119767
:102480008CEC91E09383828386E190E09583848352
:102490008091CA049091CB04A091CC04B091CD045A
:1024A00086839783A087B18788E890E093878287A7
:1024B0000E94B5298DB79EB70C960FB6F8949EBFB3
:1024C0000FBE8DBFC8010E942F051F910F91089567
:1024D000CF92DF92EF92FF920F931F93CF93DF93F0
:1024E000282F462FCEE7D4E0CE01622F0E9473043E
:1024F000CE010E944B056091190670911A068091D9
:102500001B0690911C062091020630910306409113
:102510000406509105060E94E1356B017C0120E024
:1025200030E04AE754E40E94D6351816D4F58DB74A
:102530009EB70C970FB6F8949EBF0FBE8DBF0DB718
:102540001EB70F5F1F4FADB7BEB71296DC93CE9389
:1025500011978AE391E0F801938382838EEF90E0F4
:10256000958384836091060670910706882777FD1E
:102570008095982F0E94AE349B01AC01C701B60133
:102580000E941334D80116966D937D938D939C937E
:10259000199780910A061A968C931A971B961C928B
:1025A00021C08DB79EB70C970FB6F8949EBF0FBE93
:1025B0008DBFEDB7FEB73196ADB7BEB71296DC93BF
:1025C000CE93119786ED91E0938382838EEF90E016
:1025D00095838483C682D782E086F186809109063E
:1025E000828713860E94B529EDB7FEB73C960FB6D9
:1025F000F894FEBF0FBEEDBF8EE794E00E942F055A
:10260000DF91CF911F910F91FF90EF90DF90CF90CE
:102610000895EF92FF920F931F93282F462F5EE7A6
:10262000E52E54E0F52EC701622F0E947304C70106
:102630000E944B058DB79EB70C970FB6F8949EBFBE
:102640000FBE8DBF0DB71EB70F5F1F4FEDB7FEB7A3
:10265000F282E1828CEC91E0F8019383828389EE2F
:1026600090E0958384836091C6047091C704809143
:10267000C8049091C9042091FE053091FF05409156
:102680000006509101060E94E135F80166837783C8
:102690008087918780910806828713860E94B529DA
:1026A0008DB79EB70C960FB6F8949EBF0FBE8DBF28
:1026B000C7010E942F051F910F91FF90EF90089581
:1026C000EF92FF920F931F93282F462F6EE7E62E6F
:1026D00064E0F62EC701622F0E947304C7010E94B6
:1026E0004B058DB79EB70C970FB6F8949EBF0FBEE3
:1026F0008DBF0DB71EB70F5F1F4FEDB7FEB7F2824C
:10270000E18286ED91E0F8019383828386EE90E08A
:10271000958384836091C2047091C3048091C40442
:102720009091C50420910206309103064091040661
:10273000509105060E94E135F80166837783808712
:10274000918780910906828713860E94B5298DB7EB
:102750009EB70C960FB6F8949EBF0FBE8DBFC701F3
:102760000E942F051F910F91FF90EF900895EF9217
:10277000FF920F931F93282F462F7EE7E72E74E0DA
:10278000F72EC701622F0E947304C7010E944B05F8
:102790008DB79EB70C970FB6F8949EBF0FBE8DBF36
:1027A0000DB71EB70F5F1F4FEDB7FEB7F282E18284
:1027B00086ED91E0F8019383828387EE90E0958324
:1027C00084836091DC047091DD04882777FD809517
:1027D000982F0E94AE34209102063091030640915A
:1027E0000406509105060E94E135F801668377835F
:1027F0008087918780910906828713860E94B52978
:102800008DB79EB70C960FB6F8949EBF0FBE8DBFC6
:10281000C7010E942F051F910F91FF90EF9008951F
:102820000F931F93282F462F0EE714E0C801622F45
:102830000E947304C8010E944B0580911D060E94EE
:10284000A40CC8010E942F051F910F910895EF92CB
:10285000FF920F931F93282F462FEEE7EE2EE4E012
:10286000FE2EC701622F0E947304C7010E944B0510
:102870008DB79EB70C970FB6F8949EBF0FBE8DBF55
:102880000DB71EB70F5F1F4FEDB7FEB7F282E182A3
:1028900086ED91E0F801938382838FE190E0958348
:1028A000848360911E0670911F068091200690918E
:1028B00021060E94AE342091020630910306409119
:1028C0000406509105060E94E135F801668377837E
:1028D0008087918780910906828713860E94B52997
:1028E0008DB79EB70C960FB6F8949EBF0FBE8DBFE6
:1028F000C7010E942F051F910F91FF90EF9008953F
:102900000F931F93282F462F0EE714E0C801622F64
:102910000E947304C8010E944B058DB79EB7409773
:102920000FB6F8949EBF0FBE8DBFEDB7FEB73196C0
:10293000ADB7BEB712961C930E93119780EE91E03F
:102940009383828383E890E0958384838091AC04B1
:102950009091AD04A091AE04B091AF0486839783AB
:10296000A087B18784E890E0938782878091BC0438
:102970009091BD04A091BE04B091BF048487958757
:10298000A687B7870E94B5298DB79EB740960FB628
:10299000F8949EBF0FBE8DBFC8010E942F051F91E6
:1029A0000F9108950F931F93282F462F8EE794E0E1
:1029B000622F0E9473048EE794E00E944B05809181
:1029C000C104282F30E0823030F4F4E0220F331FAE
:1029D000FA95E1F702C02150304000D000D000D07D
:1029E000EDB7FEB731960EE714E0ADB7BEB712965D
:1029F0001C930E93119780E091E09383828335833B
:102A000024830E94B5298DB79EB706960FB6F89419
:102A10009EBF0FBE8DBFC8010E942F051F910F9151
:102A200008950F931F93282F462F0EE714E0C80137
:102A3000622F0E947304C8010E944B058DB79EB798
:102A400008970FB6F8949EBF0FBE8DBFEDB7FEB7C7
:102A50003196ADB7BEB712961C930E93119782EFC5
:102A600091E0938382838FE090E0958384838091CB
:102A7000C004868317820E94B5298DB79EB7089639
:102A80000FB6F8949EBF0FBE8DBFC8010E942F05E0
:102A90001F910F9108950F931F930EE714E0C80143
:102AA00063E045E00E947304C8010E944B0500D01A
:102AB00000D0EDB7FEB71283018384E691E09483E2
:102AC00083830E94A429EDB7FEB71283018380E5BA
:102AD00091E0948383830E94A429EDB7FEB712830B
:102AE000018389E491E0948383830E94A429EDB754
:102AF000FEB71283018383E491E0948383830E9471
:102B0000A4290F900F900F900F90C8010E942F05DD
:102B10001F910F9108950F931F93282F462F0EE7B3
:102B200014E0C801622F0E947304C8010E944B0583
:102B300000D000D0EDB7FEB7128301838BE791E0A0
:102B4000948383830E94A4290F900F900F900F907D
:102B5000C8010E942F051F910F910895EF92FF92D7
:102B60000F931F93CF93DF930E944E31209127063E
:102B7000309128064091290650912A0626173707DA
:102B80004807590708F08AC10E944E316C507E4FA9
:102B90008F4F9F4F609327067093280680932906D6
:102BA00090932A060EE714E0C8010E949805C80118
:102BB00065E043E00E947304C8010E944B0500D009
:102BC00000D0EDB7FEB7128301838BED91E09483C3
:102BD00083830E94A4290F900F900F900F908091F3
:102BE0000B0690910C06892B31F080912206909172
:102BF0002306892B81F48091B8049091B9049093B5
:102C00000C0680930B068091BA049091BB049093BC
:102C10002306809322062091BA043091BB04409190
:102C2000220650912306C90184569040481759073F
:102C300024F4809126068F5F08C02C593F4F24173B
:102C400035072CF4809126068150809326068091CA
:102C50002606181614F081E003C084301CF083E0CF
:102C60008093260680912606823009F462C0833064
:102C700009F4BEC0813009F00DC100D000D0CEE70C
:102C8000D4E0EDB7FEB7D283C18382ED91E09483A7
:102C900083830E94A4298091FC050F900F900F90D0
:102CA0000F9080FF22C000D000D0EDB7FEB7D283D6
:102CB000C1838AEC91E0948383830E94A42980914C
:102CC0000B0690910C06845690400F900F900F9039
:102CD0000F902091B8043091B904281739070CF0EF
:102CE000D9C08091FC058E7F21C000D000D0EDB707
:102CF000FEB7D283C18382EC91E0948383830E94E8
:102D0000A42980910B0690910C068C599F4F0F902F
:102D10000F900F900F902091B8043091B904821752
:102D200093070CF0B7C08091FC0581608093FC058F
:102D3000B1C000D000D0CEE7D4E0EDB7FEB7D2836B
:102D4000C18388EB91E0948383830E94A4290F9030
:102D50000F900F900F9080912406882301F100D0EE
:102D600000D0EDB7FEB7D283C1838EEA91E09483A1
:102D700083830E94A42980910B0690910C068456AF
:102D800090400F900F900F900F902091B8043091C9
:102D9000B904281739071CF51092240620C000D06A
:102DA00000D0EDB7FEB7D283C18381EA91E094836E
:102DB00083830E94A42980910B0690910C068C5964
:102DC0009F4F0F900F900F900F902091B80430916B
:102DD000B904821793071CF481E08093240686E7E8
:102DE00096E06BEF73E0409124060E946D3052C074
:102DF00000D000D0AEE7EA2EA4E0FA2EEDB7FEB781
:102E0000F282E18280E991E0948383830E94A42985
:102E10008DB79EB708970FB6F8949EBF0FBE8DBFB3
:102E20000DB71EB70F5F1F4FEDB7FEB7F282E182FD
:102E300088EF91E0F801938382836091250670E02A
:102E400080E090E00E94AC3420E030E040E251E4C9
:102E50000E941334F801648375838683978386E721
:102E600090E09187808780E290E0938782870E943C
:102E7000B5298DB79EB70C960FB6F8949EBF0FBEBE
:102E80008DBF8091250690E060E873E00E94D50C2C
:102E9000809325068EE794E00E942F05DF91CF9165
:102EA0001F910F91FF90EF9008952F923F924F92B4
:102EB0005F926F927F928F929F92AF92BF92CF92CA
:102EC000DF92EF92FF920F931F93DF93CF93CDB7D3
:102ED000DEB72A970FB6F894DEBF0FBECDBF8F8343
:102EE00068870E944E31209134063091350640911A
:102EF000360650913706261737074807590708F056
:102F000051C1809138068823C9F0809387021092BE
:102F1000380680E092E090933A06809339060E944A
:102F20004E316C507E4F8F4F9F4F6093340670939D
:102F300035068093360690933706EFC0809187025E
:102F4000282E3324E090B4040091390610913A06FB
:102F50002091A10429834091C1044E8350912B06F6
:102F60005D836090CE047090CF048090D0049090E8
:102F7000D1048091250690E0409085025090860211
:102F800020912C06A22FB0E0BC83AB83B0912D061C
:102F9000BA83F090ED043A8629865C01CC24B7FC14
:102FA000C094DC2CE985FA853196FA87E987379752
:102FB0002CF041E050E05A8749871BC089859A85EB
:102FC0008330910531F1843091053CF481309105D5
:102FD00081F0029709F068C014C0A985BA85A530B0
:102FE000B105C9F1A530B10504F1169709F05CC02F
:102FF00043C0B1E0BE1508F457C00DE012E081E017
:103000005AC0E981E33009F44FC00AE112E082E0DE
:1030100052C0FE81F23008F047C02D81222309F40E
:1030200043C007E212E083E046C0C601B5010E943A
:10303000AE3420E030E040E251E40E9413349B01C2
:10304000AC01C401B3010E940C3488236CF504E385
:1030500012E084E030C04B815C814416550624F5B3
:103060005DE945165FEF5506F9F08A818823E1F4A2
:1030700001E412E085E01FC091E09E15A8F09F15C5
:1030800098F4A3E0FA1649F0B4E0FB1649F0E2E048
:10309000FE1651F40EE412E005C00AE512E002C08B
:1030A00007E612E086E007C049855A8542155305B8
:1030B00009F078CF60C010933A06009339068093E8
:1030C000380681E080932E060E944E3168517C4F75
:1030D0008F4F9F4F6093340670933506809336066A
:1030E000909337060E944E316056704F8F4F9F4F1E
:1030F00060933006709331068093320690933306C6
:1031000080912F06882321F08EE794E00E94980595
:1031100010922F0602C010922E060EE714E0C8018E
:103120006F8148850E947304C8010E944B0500D03E
:1031300000D000D0EDB7FEB73196ADB7BEB712964E
:103140001C930E93119784E792E09383828380917E
:10315000390690913A06958384830E94B529EDB78C
:10316000FEB736960FB6F894FEBF0FBEEDBFC8018E
:103170000E942F0517C010933A060093390610924B
:1031800038060E944E312091300630913106409130
:10319000320650913306261737074807590708F4B7
:1031A000BACFBBCF2A960FB6F894DEBF0FBECDBF05
:1031B000CF91DF911F910F91FF90EF90DF90CF9013
:1031C000BF90AF909F908F907F906F905F904F9047
:1031D0003F902F900895EF92FF920F931F9380914D
:1031E0003B06843009F056C09091B504943008F045
:1031F00027C1809144068917A1F1909344060E944B
:103200004E3160934006709341068093420690933E
:1032100043069091440680918802981711F5809199
:103220002F06813091F0813018F08230B1F413C054
:1032300011E010932F060E944E3161537547804074
:10324000904030F410933C0608C082E080932F0633
:1032500010923C0602C010922F068EE794E00E9466
:1032600098050E944E3120914006309141064091D0
:10327000420650914306621B730B840B950B615DF4
:1032800077408040904008F4DBC08091B504809383
:103290008802D6C0853029F480917D0290917E020B
:1032A00014C0863029F480917F02909180020DC075
:1032B000873029F4809181029091820206C0883083
:1032C00041F4809183029091840290933F06809311
:1032D0003E0680913D0620913E0630913F068823B0
:1032E00009F04AC0C901895097408F5A9440C8F4E8
:1032F0000E944E31615375478040904020F481E038
:1033000080933C060CC080913C06882341F4809158
:103310002E06882321F48EE794E00E94980582E02F
:1033200028C044E0203B340768F480912F068823AE
:1033300049F010923C068EE794E00E9498051092A6
:103340002F067EC0205B34402955324008F078C0FB
:1033500080912F06813009F473C080912E06882356
:1033600009F06EC010923C068EE794E00E9498052A
:1033700081E080932F0664C0215B344008F460C074
:103380000E944E31615375478040904008F041C023
:1033900080913C068823E9F5E0904006F0904106D4
:1033A000009142061091430688EE93E0A0E0B0E061
:1033B000E80EF91E0A1F1B1F0E944E31E616F70683
:1033C00008071907E8F581E080933C0617C01092C2
:1033D0003C068EE794E00E94980580912F0682308B
:1033E00019F410922F0603C08F5F80932F068091EF
:1033F0002F06823018F082E080932F060E944E3113
:103400006093400670934106809342069093430672
:1034100017C0E0904006F0904106009142061091DE
:10342000430688EE93E0A0E0B0E0E80EF91E0A1F24
:103430001B1F0E944E31E616F7060807190738F2DF
:103440001F910F91FF90EF90089580913B0684307B
:1034500010F00E94EB1880913C06882319F00E941E
:10346000AE1508958091E10380FF08C06091470484
:103470008091450490E070E00E94551780912F06DE
:10348000823008F0FDC1A82FB0E0FD01E552FC4FED
:10349000808185FF0BC0FD01E950FC4F6081AB507E
:1034A000BC4F8C9190E070E00E94111580912F0626
:1034B000A82FB0E0FD01E552FC4F808186FF0BC0D4
:1034C000FD01E550FC4F6081A750BC4F8C9190E00E
:1034D00070E00E94D21480912B06882309F43FC02B
:1034E00080912F06A82FB0E0FD01E552FC4F8081AE
:1034F00087FF0BC0FD01E150FC4F6081A350BC4F22
:103500008C9190E070E00E94801480912F06A82F8B
:10351000B0E0FD01E352FC4F808184FF0BC0FD0150
:10352000E95EFB4F6081AB5EBB4F8C9190E070E039
:103530000E94271480912F06A82FB0E0FD01E352CE
:10354000FC4F808183FF0BC0FD01ED5EFB4F60816E
:10355000AF5EBB4F8C9190E070E00E9410148091A0
:103560002F06A82FB0E0FD01E152FC4F808187FFBC
:103570000BC0FD01E15DFB4F6081A35DBB4F8C91F2
:1035800090E070E00E94B71380912F06A82FB0E062
:10359000FD01EF51FC4F808183FF0BC0FD01E15B1A
:1035A000FB4F6081A35BBB4F8C9190E070E00E9469
:1035B000221280912B06882309F46EC08091C104E9
:1035C000823008F469C080912F06A82FB0E0FD0179
:1035D000ED51FC4F808182FF0BC0FD01E55AFB4F8E
:1035E0006081A75ABB4F8C9190E070E00E946812F6
:1035F00080912F06A82FB0E0FD01E152FC4F8081A1
:1036000082FF0BC0FD01E55DFB4F6081A75DBB4FF5
:103610008C9190E070E00E94601380912F06A82F9B
:10362000B0E0FD01E152FC4F808183FF0BC0FD0142
:10363000ED5CFB4F6081AF5CBB4F8C9190E070E024
:103640000E94091380912F06A82FB0E0FD01E352DC
:10365000FC4F808181FF0BC0FD01E55FFB4F608166
:10366000A75FBB4F8C9190E070E00E94E0118091C9
:103670002F06A82FB0E0FD01E352FC4F808180FFB0
:103680000BC0FD01E95FFB4F6081AB5FBB4F8C91CD
:1036900090E070E00E949E1180912F06A82FB0E06C
:1036A000FD01EF51FC4F808186FF0BC0FD01E95AFF
:1036B000FB4F6081AB5ABB4F8C9190E070E00E9451
:1036C0005E1180912F06A82FB0E0FD01E552FC4F5E
:1036D000808182FF0BC0FD01E151FC4F6081A3514D
:1036E000BC4F8C9190E070E00E941E1180912F06DB
:1036F000A82FB0E0FD01E552FC4F808181FF0BC097
:10370000FD01E551FC4F6081A751BC4F8C9190E0C9
:1037100070E00E94DE1080912F06A82FB0E0FD011E
:10372000E152FC4F808184FF0BC0FD01E55CFB4F43
:103730006081A75CBB4F8C9190E070E00E949E106E
:1037400080912F06A82FB0E0FD01E152FC4F80814F
:1037500085FF0BC0FD01E15CFB4F6081A35CBB4FAB
:103760008C9190E070E00E94061080912F06A82FA7
:10377000B0E0FD01E552FC4F808183FF0BC0FD01ED
:10378000ED50FC4F6081AF50BC4F8C9190E070E0E9
:103790000E94C00F80912F06A82FB0E0FD01E152DA
:1037A000FC4F808180FF0BC0FD01E95DFB4F608114
:1037B000AB5DBB4F8C9190E070E00E946B0F8091ED
:1037C0002F06A82FB0E0FD01E552FC4F808184FF59
:1037D0000BC0FD01ED5FFB4F6081AF5FBB4F8C9174
:1037E00090E070E00E942B0F80912F06A82FB0E090
:1037F000FD01ED51FC4F808181FF18C080912406AE
:10380000FD01E35AFB4F813049F4A15ABB4F6C9143
:10381000808190E070E00E940F0E08C0A15ABB4F5B
:103820006C91808190E070E00E94620E80912F0682
:10383000A82FB0E0FD01E352FC4F808187FF0BC051
:10384000FD01ED5DFB4F6081AF5DBB4F8C9190E062
:1038500070E00E948C0D80912F06A82FB0E0FD0132
:10386000E152FC4F808186FF0BC0FD01ED5BFB4FF9
:103870006081AF5BBB4F8C9190E070E00E94310D96
:1038800008958EE794E00E9498050E944B150E94CF
:103890000A0A0895CF93DF93EC018EE794E00E942B
:1038A0006F04C817D9073CF08EE794E00E946404C7
:1038B000892B09F42397CE01DF91CF910895EF92E0
:1038C000FF920F931F93CF93DF9300912F0610E089
:1038D0008AEF90E0089F7001099FF00C189FF00C90
:1038E0001124C7010E94EF0AF801E552FC4F88231A
:1038F00019F08081816002C080818E7F80838091F9
:103900002F06C82FD0E0C70102960E94EF0ACB51C4
:10391000DC4F888380912F06C82FD0E0C701049622
:103920000E94EF0A90E00E944A1CC951DC4F888334
:1039300000912F0610E0C70188569F4F0E94EF0AA2
:10394000F801E552FC4F882319F08081806102C0A4
:1039500080818F7E808380912F06C82FD0E0C701A1
:1039600086569F4F0E94EF0ACF5FDB4F888380917E
:103970002F06C82FD0E0C70184569F4F0E94EF0A40
:1039800090E00E944A1CCD5FDB4F888300912F0698
:1039900010E0C70106960E94EF0AF801E552FC4FBD
:1039A000882319F08081826002C080818D7F8083AE
:1039B00080912F06C82FD0E0C70108960E94EF0A19
:1039C000C751DC4F888380912F06C82FD0E0C701F4
:1039D0000A960E94EF0A90E00E944A1CC551DC4FF3
:1039E000888300912F0610E0C7010C960E94EF0A11
:1039F000F801E552FC4F882319F08081846002C0F1
:103A000080818B7F808380912F06C82FD0E0C701F3
:103A10000E960E94EF0AC351DC4F888380912F06D7
:103A2000C82FD0E0C70140960E94EF0A90E00E94A4
:103A30004A1CC151DC4F888300912F0610E0C7015A
:103A400042960E94EF0AF801E552FC4F882319F0D4
:103A50008081886002C08081877F808380912F066B
:103A6000C82FD0E0C70144960E94EF0ACF50DC4F28
:103A7000888380912F06C82FD0E0C70146960E9408
:103A8000EF0A90E00E944A1CCD50DC4F88830091E1
:103A90002F0610E0C7014E960E94EF0AF801E5528A
:103AA000FC4F882319F08081806202C080818F7D65
:103AB000808380912F06C82FD0E0C70180960E9496
:103AC000EF0ACB50DC4F888380912F06C82FD0E0BF
:103AD000C70182960E94EF0A90E00E944A1CC950DA
:103AE000DC4F888300912F0610E0C70184960E9466
:103AF000EF0AF801E552FC4F882319F080818064B9
:103B000002C080818F7B808380912F06C82FD0E0F8
:103B1000C70186960E94EF0AC750DC4F88838091C8
:103B20002F06C82FD0E0C70188960E94EF0A90E0C8
:103B30000E944A1CC550DC4F888300912F0610E07C
:103B4000C7018A960E94EF0AF801E552FC4F8823CC
:103B500019F08081806802C080818F778083809196
:103B60002F06C82FD0E0C7018C960E94EF0AC350E1
:103B7000DC4F888380912F06C82FD0E0C7018E9636
:103B80000E94EF0A90E00E944A1CC150DC4F8883DB
:103B900000912F0610E0C701C0960E94EF0AF801BD
:103BA000E352FC4F882319F08081816002C080813C
:103BB0008E7F808380912F06C82FD0E0C701C296E8
:103BC0000E94EF0ACB5FDB4F888380912F06C82FBE
:103BD000D0E0C701C4960E94EF0A90E00E944A1C00
:103BE000C95FDB4F888300912F0610E0C701C6969E
:103BF0000E94EF0AF801E352FC4F882319F08081FC
:103C0000826002C080818D7F808380912F06C82FC3
:103C1000D0E0C701C8960E94EF0AC75FDB4F8883D8
:103C200080912F06C82FD0E0C701CA960E94EF0AE4
:103C300090E00E944A1CC55FDB4F888300912F06ED
:103C400010E0C701CC960E94EF0AF801E352FC4F46
:103C5000882319F08081846002C080818B7F8083FB
:103C600080912F06C82FD0E0C701CE960E94EF0AA0
:103C7000C35FDB4F888380912F06C82FD0E0C70138
:103C8000805C9F4F0E94EF0A90E00E944A1CC15F37
:103C9000DB4F888300912F0610E0C701885B9F4FA0
:103CA0000E94EF0AF801E352FC4F882319F080814B
:103CB000806102C080818F7E808380912F06C82F13
:103CC000D0E0C701865B9F4F0E94EF0ACB5EDB4FBF
:103CD000888380912F06C82FD0E0C701845B9F4F57
:103CE0000E94EF0A90E00E944A1CC95EDB4F888365
:103CF00000912F0610E0C7018E5B9F4F0E94EF0AD4
:103D0000F801E352FC4F882319F08081886002C0DB
:103D10008081877F808380912F06C82FD0E0C701E4
:103D20008C5B9F4F0E94EF0ACF5EDB4F88838091B0
:103D30002F06C82FD0E0C7018A5B9F4F0E94EF0A71
:103D400090E00E944A1CCD5EDB4F888300912F06D5
:103D500010E0C701805B9F4F0E94EF0AF801E35219
:103D6000FC4F882319F08081806202C080818F7DA2
:103D7000808380912F06C82FD0E0C7018E5A9F4FB5
:103D80000E94EF0AC75EDB4F888380912F06C82F01
:103D9000D0E0C7018C5A9F4F0E94EF0A90E00E942A
:103DA0004A1CC55EDB4F888300912F0610E0C701D7
:103DB0008A5A9F4F0E94EF0AF801E352FC4F882372
:103DC00019F08081806402C080818F7B8083809124
:103DD0002F06C82FD0E0C701885A9F4F0E94EF0AD4
:103DE000C35EDB4F888380912F06C82FD0E0C701C8
:103DF000865A9F4F0E94EF0A90E00E944A1CC15EC3
:103E0000DB4F888300912F0610E0C70182569F4F39
:103E10000E94EF0AF801E352FC4F882319F08081D9
:103E2000806802C080818F77808380912F06C82FA1
:103E3000D0E0C70180569F4F0E94EF0ACF5DDB4F55
:103E4000888380912F06C82FD0E0C7018E559F4FE1
:103E50000E94EF0A90E00E944A1CCD5DDB4F8883F0
:103E600000912F0610E0C7018E599F4F0E94EF0A64
:103E7000F801E152FC4F882319F08081816002C073
:103E800080818E7F808380912F06C82FD0E0C7016C
:103E90008C599F4F0E94EF0ACB5DDB4F8883809146
:103EA0002F06C82FD0E0C7018A599F4F0E94EF0A02
:103EB00090E00E944A1CC95DDB4F888300912F0669
:103EC00010E0C70182599F4F0E94EF0AF801E152AA
:103ED000FC4F882319F08081846002C080818B7F31
:103EE000808380912F06C82FD0E0C70180599F4F53
:103EF0000E94EF0AC75DDB4F888380912F06C82F91
:103F0000D0E0C7018E589F4F0E94EF0A90E00E94B8
:103F10004A1CC55DDB4F888300912F0610E0C70166
:103F200084579F4F0E94EF0AF801E152FC4F88230B
:103F300019F08081806802C080818F7780838091B2
:103F40002F06C82FD0E0C70182579F4F0E94EF0A6B
:103F5000C35DDB4F888380912F06C82FD0E0C70157
:103F600080579F4F0E94EF0A90E00E944A1CC15D5B
:103F7000DB4F888300912F0610E0C7018E569F4FBC
:103F80000E94EF0AF801E152FC4F882319F080816A
:103F9000826002C080818D7F808380912F06C82F30
:103FA000D0E0C7018C569F4F0E94EF0ACB5CDB4FDD
:103FB000888380912F06C82FD0E0C7018A569F4F73
:103FC0000E94EF0A90E00E944A1CC95CDB4F888384
:103FD00000912F0610E0C7018C589F4F0E94EF0AF6
:103FE000F801E152FC4F882319F08081886002C0FB
:103FF0008081877F808380912F06C82FD0E0C70102
:104000008A589F4F0E94EF0ACF5CDB4F88838091D4
:104010002F06C82FD0E0C70188589F4F0E94EF0A93
:1040200090E00E944A1CCD5CDB4F888300912F06F4
:1040300010E0C70186589F4F0E94EF0AF801E15235
:10404000FC4F882319F08081806102C080818F7EBF
:10405000808380912F06C82FD0E0C70184589F4FDE
:104060000E94EF0AC75CDB4F888380912F06C82F20
:10407000D0E0C70182589F4F0E94EF0A90E00E9453
:104080004A1CC55CDB4F888300912F0610E0C701F6
:1040900080589F4F0E94EF0AF801E152FC4F88239D
:1040A00019F08081806202C080818F7D8083809141
:1040B0002F06C82FD0E0C7018E579F4F0E94EF0AEE
:1040C000C35CDB4F888380912F06C82FD0E0C701E7
:1040D0008C579F4F0E94EF0A90E00E944A1CC15CDF
:1040E000DB4F888300912F0610E0C7018A579F4F4E
:1040F0000E94EF0AF801E152FC4F882319F08081F9
:10410000806402C080818F7B808380912F06C82FBE
:10411000D0E0C70188579F4F0E94EF0ACF5BDB4F6B
:10412000888380912F06C82FD0E0C70186579F4F04
:104130000E94EF0A90E00E944A1CCD5BDB4F88830F
:1041400000912F0610E0C7018C559F4F0E94EF0A87
:10415000F801EF51FC4F882319F08081816002C083
:1041600080818E7F808380912F06C82FD0E0C70189
:104170008A559F4F0E94EF0ACB5BDB4F888380916B
:104180002F06C82FD0E0C70188559F4F0E94EF0A25
:1041900090E00E944A1CC95BDB4F888300912F0688
:1041A00010E0C70180559F4F0E94EF0AF801EF51C0
:1041B000FC4F882319F08081846002C080818B7F4E
:1041C000808380912F06C82FD0E0C7018E549F4F67
:1041D0000E94EF0AC75BDB4F888380912F06C82FB0
:1041E000D0E0C7018C549F4F0E94EF0A90E00E94DC
:1041F0004A1CC55BDB4F888300912F0610E0C70186
:104200008A549F4F0E94EF0AF801EF51FC4F882318
:1042100019F08081886002C08081877F80838091CF
:104220002F06C82FD0E0C70188549F4F0E94EF0A85
:10423000C35BDB4F888380912F06C82FD0E0C70176
:1042400086549F4F0E94EF0A90E00E944A1CC15B77
:10425000DB4F888300912F0610E0C70184549F4FE5
:104260000E94EF0AF801EF51FC4F882319F080817A
:10427000806102C080818F7E808380912F06C82F4D
:10428000D0E0C70182549F4F0E94EF0ACF5ADB4F04
:10429000888380912F06C82FD0E0C70180549F4F9C
:1042A0000E94EF0A90E00E944A1CCD5ADB4F88839F
:1042B00000912F0610E0C701845A9F4F0E94EF0A19
:1042C000F801EF51FC4F882319F08081806402C00F
:1042D00080818F7B808380912F06C82FD0E0C7011B
:1042E000825A9F4F0E94EF0ACB5ADB4F88838091FE
:1042F0002F06C82FD0E0C701805A9F4F0E94EF0AB7
:1043000090E00E944A1CC95ADB4F888300912F0617
:1043100010E0C70180529F4F0E94EF0AF801ED5153
:10432000FC4F882319F08081846002C080818B7FDC
:10433000808380912F06C82FD0E0C7018E519F4FF8
:104340000E94EF0AC75ADB4F888380912F06C82F3F
:10435000D0E0C7018C519F4F0E94EF0A90E00E946D
:104360004A1CC55ADB4F888300912F0610E0C70115
:104370008C529F4F0E94EF0AF801ED51FC4F8823A9
:1043800019F08081826002C080818D7F808380915E
:104390002F06C82FD0E0C7018A529F4F0E94EF0A14
:1043A000C35ADB4F888380912F06C82FD0E0C70106
:1043B00088529F4F0E94EF0A90E00E944A1CC15A07
:1043C000DB4F8883DF91CF911F910F91FF90EF908A
:1043D00008954F925F927F928F929F92AF92BF9279
:1043E000CF92DF92EF92FF920F931F93DF93CF93C1
:1043F000CDB7DEB7C854D0400FB6F894DEBF0FBEBD
:10440000CDBF0EE714E0C8010E949805C80166E020
:1044100049E00E947304C8010E944B0500D000D0FF
:10442000EDB7FEB71283018386E092E09483838325
:104430000E94A4290F900F900F900F90C8010E9426
:104440002F0500D000D001E614E0EDB7FEB71283CF
:10445000018386EF91E0948383830E94A4294BEE2D
:10446000442E41E0542EEE24FF24CC24DD240F9072
:104470000F900F900F90702E012F39E0A32EB12CCA
:10448000AC0EBD1E4E010894811C911C81E694E087
:104490000E94582A982F8D3031F08D30DCF18053F6
:1044A0008230C0F530C01830A1F59981892F805332
:1044B000823078F5913311F490E801C090E08A8160
:1044C000813309F4905C8B81813309F4905E8C8197
:1044D000813309F4905F8D81813309F4985F8E8177
:1044E000813309F49C5F8F81813309F49E5F888555
:1044F000813309F49F5FF501EE0DFF1D9083089451
:10450000E11CF11C06C0F401E10FF11D90831F5F57
:1045100001C010E0F0E4EF16F104C9F48EE794E076
:10452000B601A5010E9483040894C11CD11C00D0CF
:1045300000D0EDB7FEB771820283548243820E949D
:10454000A429EE24FF240F900F900F900F90FFEFFF
:10455000CF16D10409F00CF499CFC85BDF4F0FB62A
:10456000F894DEBF0FBECDBFCF91DF911F910F91A9
:10457000FF90EF90DF90CF90BF90AF909F908F9083
:104580007F905F904F900895DF92EF92FF920F938C
:104590001F93DF93CF93CDB7DEB72A970FB6F8946A
:1045A000DEBF0FBECDBF63E0E62EF12CEC0EFD1E8C
:1045B00053E0D52EADC30E944E3160527E44804000
:1045C0009040C8F40E944E31695873418040904039
:1045D00090F01A3011F01D3031F48091F8058F5FA2
:1045E0008093F80502C01092F8058091F805833099
:1045F00011F40E94E921812F6EEE74E00E94F5060D
:10460000882311F400E07EC38091F2049091F304BA
:10461000A091F404B091F5048A3747EC940749ED72
:10462000A4074BE7B40709F45FC38B3757EC950732
:1046300059EDA5075BE7B50708F0C5C08434EBED7D
:104640009E07E0E7AE07EDE1BE0709F44DC38534F0
:10465000FBED9F07F0E7AF07FDE1BF0708F052C091
:10466000823923EA92072CEEA20724E1B20709F46B
:10467000D0C1833933EA93073CEEA30734E1B30793
:10468000C8F486314AEA940747E3A4074BE0B4072D
:1046900009F4BFC184305AE9950757EDA5075EE0DC
:1046A000B50709F4B6C18E5F9B4CA74CB94009F021
:1046B0001FC31AC38035FFED9F07FDEEAF07F8E17A
:1046C000BF0709F4E6C281352FED92072DEEA20750
:1046D00028E1B20738F488599C42AA41B64109F052
:1046E00007C3A0C18E3C48E4940747E5A4074AE10C
:1046F000B40709F4E3C184579B4EAA47BB4109F0B4
:10470000F7C287C1863AEEE09E07E2E1AE07E8E431
:10471000BE0709F489C2873AFEE09F07F2E1AF07BE
:10472000F8E4BF0740F5823523E2920726E9A207A5
:1047300026E2B20709F43FC2833533E2930736E934
:10474000A30736E2B30738F4825D924CA248BE411B
:1047500009F0CEC267C1863E55ED95075AEDA50713
:1047600053E3B50709F403C1885F9C4AAE4EB443D6
:1047700009F0BEC2B9C2823EF5E59F07FCE9AF076A
:10478000F6E6BF0709F477C2833E25E592072CE9D8
:10479000A20726E6B20738F48855964BAD4FBA44C7
:1047A00009F0A6C258C28C3E49E3940746E7A40725
:1047B0004BE6B40709F498C280569B4DAB43BE4606
:1047C00009F096C226C18A3BE4E89E07E5E2AE07FF
:1047D000EEEBBE0709F44FC28B3BF4E89F07F5E20E
:1047E000AF07FEEBBF0708F061C08E3722E19207EA
:1047F0002AE6A2072BE9B20709F40BC18F3732E191
:1048000093073AE6A3073BE9B30740F582354AEE42
:10481000940740E8A4074AE8B40709F4FAC08335CE
:104820005AEE950750E8A5075AE8B50738F4865EB2
:10483000964AA642BD4709F05BC240C18C38F5E8F4
:104840009F07F7EAAF07F8E9BF0709F437C18A56AF
:104850009E42A246B94909F04BC2E6C180323EE40D
:10486000930739EAA30731EBB30709F404C2813295
:104870004EE4940749EAA40741EBB40738F48A5799
:10488000964FA14FBD4909F033C218C18A38E7EFEE
:104890009E07E7ECAE07E8EBBE0709F4C3C0845AF5
:1048A0009040AB49BA4B09F023C21EC2843629EDB1
:1048B000920720EEA20727EDB20709F458C085360B
:1048C00039ED930730EEA30737EDB30740F5803895
:1048D00044E7940740E1A40744ECB40709F4A2C0FC
:1048E000813854E7950750E1A50754ECB50738F433
:1048F0008C569846A344B24C09F0FAC14CC1843599
:10490000FDE29F07FFEFAF07F5ECBF0709F481C099
:1049100086599543A840B24D09F0EAC14CC18E3486
:104920003DE593073EE3A30733EEB30709F471C0F7
:104930008F344DE594074EE3A40743EEB40738F4F3
:10494000865B9342A34AB24E09F0D2C1B7C0823906
:10495000E0E79E07E6E8AE07EBEFBE0709F4C4C147
:10496000825F9D4EA442BD4F09F0C2C18DC10E941D
:104970004E316093A2047093A3048093A404909397
:10498000A504D092A1048EEE94E060E170E00E9454
:10499000C9080E947B347093A7046093A6048EEE2E
:1049A00094E064E170E00E94C9080E947B34709337
:1049B000A9046093A8048EEE94E068E170E00E9480
:1049C000C9080E947B348B017093AB046093AA04E6
:1049D0006091AC047091AD048091AE049091AF04ED
:1049E00020E030E040E050E00E940C34882379F46D
:1049F000B801882777FD8095982F0E94AE34609388
:104A0000B0047093B1048093B2049093B30401E0B6
:104A100070C18091F8048093B4048091F90480936C
:104A2000B50466C18EEE94E060E070E00E94C908B3
:104A300020E030E048EC52E40E94E1350E947B34F3
:104A40007093B7046093B604693C710520F010922E
:104A5000B7041092B60480911205909113059093BB
:104A6000B9048093B8048091140590911505909332
:104A7000BB048093BA048091180590911905909316
:104A80007E0280937D0280911C0590911D0590937C
:104A9000800280937F0280911E0590911F05909364
:104AA00082028093810280912005909121059A8352
:104AB000898390938402809383021AC16091F804E1
:104AC0007091F9048091FA049091FB040E94AE3435
:104AD00020E836E948E15BE40E9413346093AC04BB
:104AE0007093AD048093AE049093AF046091FC0486
:104AF0007091FD048091FE049091FF04D7016C93A6
:104B000011967C93119712968C93129713969C93FF
:104B10000E94AE3420E836E948E15BE40E94133499
:104B20006093BC047093BD048093BE049093BF0453
:104B300080911D058093C00480911C058093C10461
:104B40008EEE94E060E170E00E94C9086093B004CA
:104B50007093B1048093B2049093B3048EEE94E00A
:104B600068E070E00E94C9086093C2047093C304B7
:104B70008093C4049093C5048EEE94E064E170E0E9
:104B80000E94C9086093C6047093C7048093C80448
:104B90009093C904ADC08EEE94E068E070E00E948E
:104BA000C90890586093CA047093CB048093CC04D6
:104BB0009093CD049DC08EEE94E060E070E00E9482
:104BC000C9086093CE047093CF048093D00490936F
:104BD000D1048EEE94E064E070E00E94C90820E009
:104BE00030E048EC52E40E94E1350E947B3470933F
:104BF000D3046093D2048EEE94E064E170E00E94EE
:104C0000C9080E947B347093D5046093D4048EEE5F
:104C100094E068E170E00E94C9080E947B347093C0
:104C2000D7046093D60464C08EEE94E064E070E034
:104C30000E94C9080E947B34882777FD8095982FB1
:104C40000E94AE346093D8047093D9048093DA0440
:104C50009093DB044DC08EEE94E068E070E00E941B
:104C6000C9080E947B34709561957F4F7093DD0475
:104C70006093DC043DC0809158058093DE048091F0
:104C800059058093DF0434C08091F8048093E004D8
:104C90002FC08EEE94E060E070E00E94C90860933F
:104CA000E1047093E2048093E3049093E4048EEEB5
:104CB00094E064E070E00E94C9086093E50470939A
:104CC000E6048093E7049093E8048EEE94E068E0B5
:104CD00070E00E94C9086093E9047093EA0480932D
:104CE000EB049093EC0404C0809104058093ED04E0
:104CF00000E08091EF04823229F48EEE94E063E2CA
:104D00000E94E1098EEB90E00E94B531002331F55D
:104D100081E694E00E94282A18161906F4F481E628
:104D200094E00E94582A182F8091A104882309F04A
:104D300062CC41CC1092A10401E0802F90E02A9631
:104D40000FB6F894DEBF0FBECDBFCF91DF911F919C
:104D50000F91FF90EF90DF90089500E02091A20462
:104D60003091A3044091A4045091A504205F384DD4
:104D70004F4F5F4F2F83388749875A870E944E31A4
:104D80002F81388549855A852617370748075907DF
:104D900088F2D3CFEF92FF920F931F9380912D064D
:104DA000882351F081E00E94EA3264E070E00E94C2
:104DB0001B376093FD053CC081E00E94EA32AA27C0
:104DC00097FDA095BA2FBC01CD010E94AE342DEC09
:104DD0003CEC4CE45EE30E94E13520E030E040E84A
:104DE0005EE30E94E1357B018C016091FD0570E07E
:104DF000882777FD8095982F0E94AE342DEC3CECEF
:104E00004CE45FE30E94E1359B01AC01C801B701AE
:104E10000E9446330E94803420914806621730F089
:104E200030914706262F361708F4232F2093FD05CF
:104E30001F910F91FF90EF90089583E00E94E73259
:104E400008951F93CF93DF9385E090E06CE070E0CE
:104E50000E948B1568EE73E080E090E00E945C3168
:104E600081E694E00E94A52AC0E0D0E010E0CE01E7
:104E70006DE171E00E941B37892BA9F41F5E8EE75C
:104E800094E0612F4CE00E9473048EE794E00E944E
:104E90004B058EE794E06EEE0E947B058EE794E072
:104EA0000E942F05105161E070E080E090E00E94C8
:104EB0005C31219687E0C13DD807C9F6DF91CF91DB
:104EC0001F91089586E061E00E94933208950F9348
:104ED0001F9386E061E00E94543201E614E0C801AD
:104EE00040E051EE60E070E00E94C6291093780621
:104EF000009377060E9462278EE794E00E94D10516
:104F00000E94411C64EF71E080E090E00E945C31FF
:104F100083EF93E00E94EF0A813011F00E94000DB0
:104F20000E94600A10922F0607C00E945F1C8091A9
:104F30002F068F5F80932F0680912F068230A8F373
:104F400010922F060E9421270E941D2780E994E0DD
:104F500068E379E224E630E040E050E000E00E94BF
:104F600079308EE794E00E94980580E994E00E94F1
:104F7000DF301F910F9108952F923F924F925F92D1
:104F80006F927F928F929F92AF92BF92CF92DF9259
:104F9000EF92FF920F931F93DF93CF9300D000D037
:104FA000CDB7DEB780912B06882309F4E1C0E090ED
:104FB0005006F09051060091520610915306C80118
:104FC000B7019F7725E33AEF4EE85CE30E94E135B5
:104FD0000E94103469837A838B839C83C801B70154
:104FE0002091AC043091AD044091AE045091AF04D7
:104FF0000E9445331B012C019F7720EC3BE649EDD5
:1050000057E40E94E1355B016C0160915406709198
:10501000550680915606909157062091BC04309118
:10502000BD044091BE045091BF040E9445333B0132
:105030004C019F7720EC3BE649ED57E40E94E135B7
:1050400029813A814B815C810E94E1357B018C0191
:10505000C601B501A60195010E94E1355B016C0115
:10506000C801B701A80197010E94E1359B01AC017D
:10507000C601B5010E9446330E9468360E947B3407
:1050800060931E0670931F0680932006909321065E
:1050900060E070E080E89FE329813A814B815C8188
:1050A0000E9413349B01AC01C201B1010E94E135A1
:1050B00097FA909497F89094A40193010E94B933C1
:1050C00020EE3EE245E652E40E94E13520E030E089
:1050D00044EB52E40E9446330E947B349B01AC01B6
:1050E00097FF04C028593E4F4F4F5F4FCA01B90187
:1050F000645B70408040904097FF06C0CA01B901D0
:105100006C547F4F8F4F9F4F0E94AE342091B0045C
:105110003091B1044091B2045091B3040E944533E0
:105120000E947B3497FF04C068597E4F8F4F9F4F7A
:105130000E94AE3420E030E044EB53E40E9413348C
:1051400020E030E040E851E40E94E1350E9444361E
:1051500020E030E040E85FE30E9446330E94803464
:1051600060931D06613108F46CC010921D0669C081
:105170008091C104823008F464C08091C0048530FD
:1051800008F45FC0A09058068DE18A1508F459C054
:10519000E090C204F090C3040091C4041091C504CF
:1051A0006091590670915A0680915B0690915C0659
:1051B000A80197010E9445339F7720E030E040E04E
:1051C0005FE30E94D63518165CF410925806E09200
:1051D0005906F0925A0600935B0610935C0631C0A4
:1051E0008A2D8F5F809358068E3159F58091AC04DB
:1051F0009091AD04A091AE04B091AF04809350069D
:1052000090935106A0935206B09353068091BC042C
:105210009091BD04A091BE04B091BF048093540648
:1052200090935506A0935606B0935706E0925D06FC
:10523000F0925E0600935F061093600681E0809313
:105240002B060F900F900F900F90CF91DF911F9131
:105250000F91FF90EF90DF90CF90BF90AF909F9015
:105260008F907F906F905F904F903F902F90089518
:10527000CF92DF92EF92FF920F931F930E94CA2664
:105280008091FD05282F30E030938602209385021F
:1052900080912D06882359F50091480610E0201BC7
:1052A000310BB901882777FD8095982F0E94AE3485
:1052B0006B017C016091470670E0601B710B8827D1
:1052C00077FD8095982F0E94AE349B01AC01C701F9
:1052D000B6010E94133420E030E048EC52E40E9412
:1052E000E1350E947B347093860260938502809141
:1052F0008502909186028D599F4F34F48DE99FEF7E
:1053000090938602809385020E9452080E94F50ABB
:105310008EE794E00E94BC270E94251A1F910F91EE
:10532000FF90EF90DF90CF9008950E94C422892BC8
:1053300019F00E943829089580E994E00E94C7304E
:1053400008958FEF9FE70895DF93CF93CDB7DEB732
:10535000FE0139968D819E8161E04F8158859F01C4
:105360000E94452CCF91DF910895DF93CF93CDB765
:10537000DEB7FE0139968D819E8160E04F815885B0
:105380009F010E94452CCF91DF9108950F931F93A9
:10539000DC01ED91FC910288F389E02D20E030E002
:1053A00000E010E009951F910F9108958F92AF9240
:1053B000CF92EF92FF920F931F93DF93CF93CDB7CE
:1053C000DEB7FC011382128288EE93E0A0E0B0E029
:1053D00084839583A683B78384EC93E09183808351
:1053E0005587448737872687118B008BF38AE28A9B
:1053F000C48AA58A868A70E0CB0123E0880F991FB2
:105400002A95E1F79C012B59394F308F278B83590F
:10541000994F928F818F81E090E002C0880F991F91
:105420006A95E2F720917506282B20937506CF0127
:1054300040E051EE60E070E00E94C629CF91DF911C
:105440001F910F91FF90EF90CF90AF908F900895A4
:10545000FC01838D882319F42FEF3FEF0DC00788DF
:10546000F08DE02D2081318182819381281B390BC1
:105470008481958128233923C9010895FC01838DF6
:10548000882319F42FEF3FEF11C0018CF28DE02D2E
:105490002081318182819381281B390B20953095A1
:1054A00084819581282339232F5F3F4FC9010895B7
:1054B000FC01838D882361F0A789B08D2D913C91EB
:1054C000119712968D919C9113972817390721F403
:1054D0004FEF5FEFCA01089512968D919C9113973B
:1054E0001696ED91FC911797E80FF91F40811296DF
:1054F0008D919C911397019614962D913C9115973F
:105500008223932313969C938E93129750E0E2CFBD
:10551000FC01838D882351F00788F08DE02D2081D8
:105520003181828193812817390721F42FEF3FEFD2
:10553000C9010895828193810680F781E02DE80FEB
:10554000F91F8081282F30E0F3CFDC015796ED91D1
:10555000FC91589782819381918380835996ED9134
:10556000FC915A9780819181938382830895DC0115
:105570005B968C915B978823A9F15996ED91FC91EC
:105580005A97208131812F5F3F4F84819581282355
:1055900039235C968C915C97882329F082819381D2
:1055A00028173907F9F08281938128173907D9F331
:1055B000808191810680F781E02DE80FF91F6083DB
:1055C0005996ED91FC915A97318320835296ED9133
:1055D000FC915397808156969C91892B808321E082
:1055E00030E002C020E030E0C9010895CF93DF939E
:1055F000EC011B821A828A819B81998388831D8298
:105600001C828E819F81009721F00E94C5031F821A
:105610001E82DF91CF9108950F931F938C01DC01BF
:105620005296ED91FC915397208156968C91569706
:1056300055969C915597892B809582238083579608
:105640008D919C9158970E94F62AF801818D928D38
:105650000E94F62AD8015B961C921F910F91089523
:105660000F931F93CF93DF938C01FC01138212825F
:10567000828193819183808341E0A1E0B0E001C009
:105680004F5FFD01042E02C0EE0FFF1F0A94E2F7E8
:105690009B0182E06130780710F020E032E0E217F1
:1056A000F30770F3C1E0D0E002C0CC0FDD1F4A95D4
:1056B000E2F72197F801268137812115310541F064
:1056C000848195818C179D0789F0C9010E94C503CB
:1056D000F801D583C483CE0101960E941B039C016F
:1056E000F8019783868380E0232B09F081E0DF9126
:1056F000CF911F910F910895AF92BF92CF92DF92F9
:10570000EF92FF920F931F93CF93DF937C015A0187
:105710006B01E901DC015B968C915B978823F1F0CA
:105720002115310539F45796ED91FC915897C481B4
:10573000D58121960115110549F4D7015996ED91AE
:10574000FC915A97048115810F5F1F4FD701ED918E
:10575000FC910088F189E02DC7010995F70187893F
:10576000908D209711F4C0E8D0E0BE010E94302B4C
:10577000882381F0D70159968D919C915A970115F4
:10578000110511F400E110E0B8010E94302B8823CC
:1057900009F04DC0D701ED91FC910088F189E02D11
:1057A000C701099567C0D7015096ED91FC915197BB
:1057B000B0E0AB16B1EEBB06B0E0CB06B0E0DB0666
:1057C00009F454C081E090E0D70154960C9002C0D7
:1057D000880F991F0A94E2F7808360E079E08DE3F7
:1057E00090E0A60195010E94503721503040404082
:1057F0005040CA01B90122E030E040E050E00E9490
:105800005037D7011C96ED91FC911D9730831E9661
:10581000ED91FC911F972083D7015296ED91FC9159
:105820005397808155969C91892B808323C0D70103
:105830005996ED91FC915A9713821282828193813D
:10584000918380835796ED91FC9158971382128231
:10585000828193819183808381E05B968C931A147B
:105860001B041C041D040CF49ECFD6CF108220E133
:1058700030E0C7CFDF91CF911F910F91FF90EF9054
:10588000DF90CF90BF90AF9008952F923F924F92AC
:105890005F926F927F928F929F92AF92BF92CF92C0
:1058A000DF92EF92FF920F931F93DF93CF93CDB7C9
:1058B000DEB764970FB6F894DEBF0FBECDBF3C01D4
:1058C000688B5A8B498B69011C01AE014F5F5F4F9A
:1058D0005C8B4B8BE989FA89488940FD659140FFD3
:1058E0006191FA8BE98B662309F4D7C3653249F4D9
:1058F00040FD859140FF8191FA8BE98B8532B1F4AF
:105900000CC06A3051F4D301ED91FC910190F0810B
:10591000E02DC1016DE009956AE0D301ED91FC91A4
:105920000190F081E02DC1010995D4CF982F10E0AE
:10593000882499241032B0F49B3269F09C3228F408
:10594000903251F0933271F40BC09D3239F09033A4
:1059500049F4116028C01260146025C0186023C08B
:10596000106121C017FD2BC0892F80538A3078F435
:1059700016FF06C0BAE09B9E902C1124980E13C00F
:10598000EAE08E9E802C1124880E10620CC09E329C
:1059900021F416FD82C3106406C09C3611F4106811
:1059A00002C0983661F4E989FA89488940FD9591E9
:1059B00040FF9191FA8BE98B992309F0BBCF892F96
:1059C0008554833020F4812F8061905E07C0892F39
:1059D0008556833008F0E6C1812F8F7E86FD02C098
:1059E00076E0972E6FE3F62EF822953619F450E400
:1059F000F52A07C0963619F480E8F82A02C09110FB
:105A00009A94F7FE0BC09BE3991520F427E05CE322
:105A1000B52E0DC0B92CB39427E009C0A7E0A91595
:105A200020F447E0942E27E001C0292DBB24F60185
:105A30003496FD87EC87D6016D917D918D919C9177
:105A4000AE014F5F5F4F0B2D0E9443026C01098135
:105A5000E02FF0E0FF87EE8700FF05C0FE85F3FD35
:105A600002C01DE209C0F1FE02C01BE205C0F2FC4B
:105A700002C010E001C010E28E859F858C7090708E
:105A8000892B09F444C0112311F483E001C084E0A0
:105A9000881510F088240EC0881AF3FC0BC0D301BF
:105AA000ED91FC910190F081E02DC10160E209953A
:105AB0008A94A9F7112349F0D301ED91FC9101904B
:105AC000F081E02DC101612F0995BE85B3FF03C0B0
:105AD0000FE013E012C003E113E00FC0E114F10482
:105AE00009F06052D301ED91FC910190F081E02D1D
:105AF000C10109950F5F1F4F05C0EF2CFF24B0E1D6
:105B0000EB22FF24F8016491662341F748C1F7FEB8
:105B100013C0BC0CFE85F4FF04C08A81813309F4F4
:105B2000BA941B141CF0BB24B3942DC048E04B1551
:105B300050F538E0B32E27C0F6FC25C0892D90E043
:105B40008C159D054CF05CEFC5165FEFD50624F073
:105B500080E8F82A01C09A94992049F0E2E0F0E048
:105B6000EC0FFD1FE90DF11D80818033A1F3F7FEDD
:105B70000AC0B92CB394892D90E0C816D90614F048
:105B8000992401C09C18F7FC03C025E030E009C04F
:105B90001C141D041CF021E030E003C096012F5FAF
:105BA0003F4F112311F02F5F3F4F992029F0892D8E
:105BB00090E00196280F391F882D90E028173907AB
:105BC00014F0882401C0821A4F2C5524C201897018
:105BD0009070892B59F00CC0D301ED91FC9101908C
:105BE000F081E02DC10160E209958A948820A1F737
:105BF000112349F0D301ED91FC910190F081E02D4A
:105C0000C101612F099543FE0BC00CC0D301ED917A
:105C1000FC910190F081E02DC10160E309958A9427
:105C20008820A1F7F7FE51C08601D7FE02C000E030
:105C300010E076010894E11CF11CE01AF10AE1E0A1
:105C4000F0E0EC0FFD1FEE0EFF1E26014B18510871
:105C5000892D90E0AA24BB24A81AB90AFFEF0F3FB0
:105C60001F0749F4D301ED91FC910190F081E02DE3
:105C7000C1016EE20995C016D10634F040165106F6
:105C80001CF4F701608101C060E3015010400894EA
:105C9000E11CF11C0A151B054CF0D301ED91FC91A0
:105CA0000190F081E02DC1010995D8CF0C151D059B
:105CB00041F48A81863320F4853319F4BE85B4FF1C
:105CC00061E3D301ED91FC9165C06A81613309F014
:105CD0000F7ED301ED91FC910190F081E02DC10187
:105CE00009959920E1F0D301ED91FC910190F081AB
:105CF000E02DC1016EE2099512E0E1E0F0E0EC0F69
:105D0000FD1FE10FF11D60811F5FD301ED91FC913B
:105D10000190F081E02DC10109959A9471F7D301AA
:105D2000ED91FC910190F081E02D44FC02C065E60C
:105D300001C065E4C1010995D7FC05C0C114D104B7
:105D400041F404FF06C0D094C194D108D3946DE20D
:105D500001C06BE2D301ED91FC910190F081E02D47
:105D6000C101099560E305C06F5FE6EFFFEFCE0E5E
:105D7000DF1EFAE0CF16D104BCF7D301ED91FC9100
:105D80000190F081E02DC1010995D301ED91FC91C5
:105D90006C2D605D0190F081E02DC1010995CC84EE
:105DA000DD8478C1933631F0933799F0933509F05B
:105DB00061C023C0F601808189835E010894A11C23
:105DC000B11C42E050E0C40ED51E21E0E22EF12CC1
:105DD00012C0D601AD90BC9016FD03C06FEF7FEFEF
:105DE00002C0692D70E0E2E0F0E0CE0EDF1EC501DA
:105DF0000E9428047C011F7713C0D601AD90BC908F
:105E000016FD03C06FEF7FEF02C0692D70E0E2E086
:105E1000F0E0CE0EDF1EC5010E941D047C0110685B
:105E200013FF0BC023C0D301ED91FC910190F081D1
:105E3000E02DC10160E209958A94882D90E0E81672
:105E4000F90688F313C0F50117FD659117FF6191FD
:105E50005F01D301ED91FC910190F081E02DC10132
:105E6000099581108A940894E108F108E114F1047D
:105E700051F710C1943611F0993699F517FF0AC001
:105E8000F601208131814281538184E090E0C80E87
:105E9000D91E0CC0D6018D919C919C01442737FDE1
:105EA0004095542FE2E0F0E0CE0EDF1E9FE6F92E83
:105EB000F12257FF09C050954095309521953F4FED
:105EC0004F4F5F4FF0E8FF2ACA01B901AE014F5FA3
:105ED0005F4F2AE030E00E94E501E82E4B89E41A8A
:105EE00041C0953721F41F7E2AE030E01CC0197FA5
:105EF0009F3661F0903720F4983509F0CEC00FC07E
:105F0000903739F0983709F0C8C004C028E030E075
:105F10000AC0106114FD146020E130E004C014FDDB
:105F2000166020E132E017FF08C0D6016D917D9127
:105F30008D919C91E4E0F0E008C0D6018D919C9198
:105F4000BC0180E090E0E2E0F0E0CE0EDF1EAE01AA
:105F50004F5F5F4F0E94E501E82EFB89EF1A8FE744
:105F6000F82EF122F6FE0BC04EEFF422E91438F4BD
:105F7000F4FE07C0F2FC05C05FEEF52202C01E2D44
:105F800001C0192DF4FE0DC0FE01EE0DF11D808142
:105F9000803319F489EEF82208C01F5FF2FE05C0B5
:105FA00003C08F2D867809F01F5F0F2DF3FC18C0FA
:105FB000F0FE13C0181510F09E2C0FC09E2C980CEC
:105FC000911A182D0AC0D301ED91FC910190F08136
:105FD000E02DC10160E209951F5F1815A0F304C010
:105FE000181510F4811A01C0882404FF17C0D301CA
:105FF000ED91FC910190F081E02DC10160E30995E4
:1060000002FF29C0D301ED91FC910190F081E02DB8
:1060100001FD02C068E712C068E510C0802F8678D5
:10602000D1F001FF02C06BE201C060E2F7FC6DE25B
:10603000D301ED91FC910190F081E02DC101099512
:106040000AC0D301ED91FC910190F081E02DC101D6
:1060500060E309959A94E914A0F3EA94D301ED91D1
:10606000FC91A1E0B0E0AC0FBD1FAE0DB11D0190E1
:10607000F081E02DC1016C910995EE2071F70AC005
:10608000D301ED91FC910190F081E02DC10160E21E
:1060900009958A948820A1F71DCC64960FB6F894D0
:1060A000DEBF0FBECDBFCF91DF911F910F91FF904B
:1060B000EF90DF90CF90BF90AF909F908F907F90A8
:1060C0006F905F904F903F902F900895F999FECF79
:1060D00072BD61BDF89A80B50895F999FECF1FBAD7
:1060E00072BD61BD40BD0FB6F894FA9AF99A0FBE21
:1060F00008950F93FC016115710511F480E011C042
:106100002183328343835483728761870170000F38
:10611000000F000F8081877F802B82608B7F8083C0
:1061200081E00F910895CF93DF93EC010E944E31EF
:106130009B01AC018D819E81AF81B88528173907FD
:106140004A075B0728F4888184FD02C060E00DC027
:1061500089819A81AB81BC81820F931FA41FB51FD7
:106160008D839E83AF83B88761E0222757FD2395F7
:10617000332744275527922F91709295907F8881DD
:106180008F7E892B8883862FDF91CF910895CF93BF
:10619000DF93EC01888182FF0FC0CE010E94933013
:1061A000882351F0E985FA85309709F009958881AF
:1061B00083FF02C08B7F8883DF91CF910895CF93B7
:1061C000DF93EC0189859A85892BE1F089819A8199
:1061D000AB81BC810097A105B105A1F00E944E31B1
:1061E00029813A814B815C81260F371F481F591F37
:1061F0002D833E834F835887888184608F7E888378
:1062000081E001C080E0DF91CF9108951F920F924D
:106210000FB60F9211242F933F938F939F93AF93B9
:10622000BF9380917D0690917E06A0917F06B091EC
:106230008006309181060196A11DB11D232F2D5F8F
:106240002D3720F02D570196A11DB11D20938106F9
:1062500080937D0690937E06A0937F06B093800680
:106260008091790690917A06A0917B06B0917C0688
:106270000196A11DB11D8093790690937A06A09393
:106280007B06B0937C06BF91AF919F918F913F9118
:106290002F910F900FBE0F901F9018958FB7F89405
:1062A00020917D0630917E0640917F0650918006B8
:1062B0008FBFB901CA0108959B01AC017FB7F89463
:1062C0008091790690917A06A0917B06B0917C0628
:1062D00066B5A89B05C06F3F19F00196A11DB11DC1
:1062E0007FBFBA2FA92F982F8827860F911DA11D38
:1062F000B11D62E0880F991FAA1FBB1F6A95D1F7D5
:10630000BC012DC0FFB7F8948091790690917A0670
:10631000A0917B06B0917C06E6B5A89B05C0EF3F37
:1063200019F00196A11DB11DFFBFBA2FA92F982FFB
:1063300088278E0F911DA11DB11DE2E0880F991FC6
:10634000AA1FBB1FEA95D1F7861B970B885E934067
:10635000C8F2215030404040504068517C4F2115D8
:1063600031054105510571F60895019739F0880FFF
:10637000991F880F991F02970197F1F70895789454
:1063800084B5826084BD84B5816084BD85B582603A
:1063900085BD85B5816085BDEEE6F0E080818160D8
:1063A0008083E1E8F0E010828081826080838081D8
:1063B00081608083E0E8F0E0808181608083E1EBB0
:1063C000F0E0808184608083E0EBF0E08081816098
:1063D0008083EAE7F0E0808184608083808182604E
:1063E0008083808181608083808180688083109237
:1063F000C10008951F920F920FB60F9211242F9390
:106400003F934F935F936F937F938F939F93AF933C
:10641000BF93EF93FF938091820690918306892B1F
:1064200029F0E0918206F09183060995FF91EF91A2
:10643000BF91AF919F918F917F916F915F914F919C
:106440003F912F910F900FBE0F901F9018951F92A4
:106450000F920FB60F9211242F933F934F935F9398
:106460006F937F938F939F93AF93BF93EF93FF931C
:106470008091840690918506892B29F0E09184060D
:10648000F09185060995FF91EF91BF91AF919F9192
:106490008F917F916F915F914F913F912F910F90CD
:1064A0000FBE0F901F901895CF93DF93482F50E0A9
:1064B000CA01875B9C4FFC0134914B5C5C4FFA0135
:1064C0008491882369F190E0880F991FFC01E95EAF
:1064D000FC4FA591B491FC01EF5DFC4FC591D491A7
:1064E000662351F42FB7F8948C91932F90958923BC
:1064F0008C93888189230BC0623061F42FB7F894A4
:106500008C91932F909589238C938881832B8883FA
:106510002FBF06C09FB7F8948C91832B8C939FBF9D
:10652000DF91CF910895482F50E0CA01835A9C4FC4
:10653000FC012491CA01875B9C4FFC0194914B5C48
:106540005C4FFA013491332309F440C0222351F106
:10655000233071F0243028F42130A1F0223011F5DD
:1065600014C02630B1F02730C1F02430D9F404C073
:10657000809180008F7703C0809180008F7D809311
:10658000800010C084B58F7702C084B58F7D84BD34
:1065900009C08091B0008F7703C08091B0008F7DDB
:1065A0008093B000E32FF0E0EE0FFF1FEF5DFC4F94
:1065B000A591B4912FB7F894662321F48C9190950E
:1065C000892302C08C91892B8C932FBF08958093CF
:1065D00089020895982F8E3008F09E509770809110
:1065E00089028295880F880F807C892B80937C009C
:1065F00080917A00806480937A0080917A0086FD91
:10660000FCCF2091780040917900942F80E030E019
:10661000282B392BC9010895CF92DF92EF92FF9278
:106620000F931F93CF93DF937C016B018A01C0E02E
:10663000D0E00FC0D6016D916D01D701ED91FC91B5
:106640000190F081E02DC7010995C80FD91F0150B5
:1066500010400115110571F7CE01DF91CF911F9107
:106660000F91FF90EF90DF90CF900895CF93DF933D
:106670000E94BF310E946727C0E0D0E00E949529A8
:106680002097E1F30E940000F9CF5058BB27AA27BA
:106690000ED041C201D230F006D220F031F49F3F3B
:1066A00011F41EF4C0C10EF4E095E7FBB6C1E92F6A
:1066B00054D280F3BA17620773078407950718F05E
:1066C00071F49EF56CC20EF4E0950B2EBA2FA02D3E
:1066D0000B01B90190010C01CA01A0011124FF278F
:1066E000591B99F0593F50F4503E68F11A16F0408A
:1066F000A22F232F342F4427585FF3CF4695379589
:106700002795A795F0405395C9F77EF41F16BA0B4D
:10671000620B730B840BBAF09150A1F0FF0FBB1FFB
:10672000661F771F881FC2F70EC0BA0F621F731F44
:10673000841F48F4879577956795B795F7959E3FA1
:1067400008F0B3CF9395880F08F09927EE0F97952F
:1067500087950895A1D158F080E891E009F49EEF63
:10676000A2D128F040E851E059F45EEF09C05BC1C6
:1067700016C2E92FE078F1D168F3092E052AC1F39A
:10678000261737074807590738F00E2E07F8E02577
:1067900069F0E025E0640AC0EF6307F8009407FAA7
:1067A000DB01B9019D01DC01CA01AD01EF934AD0C3
:1067B000B2D10AD05F91552331F02BED3FE049E48F
:1067C00050FD49EC63CF0895DF93DD27B92FBF77E4
:1067D00040E85FE31616170648075B0710F4D92F49
:1067E000E9D19F938F937F936F93BCD2E8E6F0E05B
:1067F0001DD191D12F913F914F915F91EED1DD232A
:1068000049F09058A2EA2AED3FE049EC5FE3D078E6
:106810005D274DDFDF917FC1DCD008F481E0089572
:106820004AD1E39589C10CD076C13DD140F034D135
:1068300030F021F45F3F19F0F0C05111B1C1F3C045
:106840008CD198F39923C9F35523B1F3951B550BBC
:10685000BB27AA2762177307840738F09F5F5F4F33
:10686000220F331F441FAA1FA9F333D00E2E3AF074
:10687000E0E830D091505040E695001CCAF729D08E
:10688000FE2F27D0660F771F881FBB1F26173707DD
:106890004807AB07B0E809F0BB0B802DBF01FF270D
:1068A00093585F4F2AF09E3F510568F0B6C078C1FB
:1068B0005F3FECF3983EDCF3869577956795B79547
:1068C000F7959F5FC9F7880F911D9695879597F962
:1068D0000895E1E0660F771F881FBB1F62177307DB
:1068E0008407BA0720F0621B730B840BBA0BEE1FF0
:1068F00088F7E095089504D06894B11151C10895C6
:1069000034D188F09F5790F0B92F9927B751A0F054
:10691000D1F0660F771F881F991F1AF0BA95C9F733
:1069200012C0B13081F03BD1B1E0089538C1672F7A
:10693000782F8827B85F39F0B93FCCF386957795E3
:106940006795B395D9F73EF49095809570956195CC
:106950007F4F8F4F9F4F0895E89409C097FB3EF4F7
:1069600090958095709561957F4F8F4F9F4F99239C
:10697000A9F0F92F96E9BB279395F695879577951A
:106980006795B795F111F8CFFAF4BB0F11F460FFDA
:106990001BC06F5F7F4F8F4F9F4F16C0882311F032
:1069A00096E911C0772321F09EE8872F762F05C046
:1069B000662371F096E8862F70E060E02AF09A95E1
:1069C000660F771F881FDAF7880F9695879597F9D6
:1069D0000895990F0008550FAA0BE0E8FEEF161670
:1069E0001706E807F907C0F012161306E407F507C3
:1069F00098F0621B730B840B950B39F40A2661F037
:106A0000232B242B252B21F408950A2609F4A140D9
:106A1000A6958FEF811D811D089597F99F6780E8E6
:106A200070E060E008959FEF80EC0895DF93CF93CE
:106A30001F930F93FF92EF92DF927B018C0168947A
:106A400005C0DA2EEF01C9D0FE01E894A591259189
:106A5000359145915591AEF3EF0129DEFE01970185
:106A6000A801DA9479F7DF90EF90FF900F911F91D2
:106A7000CF91DF9108959F938F937F936F93FF93AF
:106A8000EF939B01AC019DD0EF91FF91CFDF2F9150
:106A90003F914F915F9195C000240A9416161706F6
:106AA00018060906089500240A94121613061406FF
:106AB00005060895B8CF59D0E8F3E894EFEFBB2767
:106AC0003FE048EC5FE76B3D73078407950708F1EB
:106AD000FF279F57B25A6A4D7F40894CF04032F4ED
:106AE000BE556542704F8643FF4F0894EE1F91508C
:106AF00030F0BB0F661F771F881FFF1FEBCF9EE78D
:106B0000882332F0BB0F661F771F881F9A95C1F745
:106B10009395E09565C1092E0394000C11F4882328
:106B200052F0BB0F40F4BF2B11F460FF04C06F5F45
:106B30007F4F8F4F9F4F0895EF93E0FF06C0A2EA6B
:106B40002AED3FE049EC5FEBB2DDE5DF0F90039407
:106B500001FC9058E5E9F0E08ECF57FD9058440FC6
:106B6000551F59F05F3F71F04795880F97FB991FAC
:106B700061F09F3F79F08795089512161306140669
:106B8000551FF2CF4695F1DF08C0161617061806F6
:106B9000991FF1CF86957105610508940895E894D1
:106BA000BB2766277727CB0197F9089512DF08F4F2
:106BB0008FEF08959B01AC0160E070E080E89FE3F7
:106BC00032CE0BD0A8CF68DF28F06DDF18F0952308
:106BD00009F023CF28CF1124E3CFBFDFA0F3959F87
:106BE000D1F3950F50E0551F629FF001729FBB27B4
:106BF000F00DB11D639FAA27F00DB11DAA1F649F60
:106C00006627B00DA11D661F829F2227B00DA11D12
:106C1000621F739FB00DA11D621F839FA00D611D98
:106C2000221F749F3327A00D611D231F849F600DB9
:106C3000211D822F762F6A2F11249F5750408AF0F2
:106C4000E1F088234AF0EE0FFF1FBB1F661F771F7E
:106C5000881F91505040A9F79E3F510570F0DDCE3E
:106C60009FCF5F3FECF3983EDCF386957795679571
:106C7000B795F795E7959F5FC1F7FE2B880F911D9C
:106C80009695879597F9089570DFE0F09E37D8F0D4
:106C90009639B8F49E3848F4672F782F8827985F84
:106CA000F9CF86957795679593959539D0F3B62F5B
:106CB000B1706B0F711D811D20F4879577956795D5
:106CC000939573C08DC06CCF11F40EF4ACCE88C018
:106CD0004CDFD0F39923D9F3CEF39F57550B87FFA1
:106CE0008FD056959795B0E020F4660F771F881FD8
:106CF000BB1F1F930F9300249001A0018001F0019E
:106D0000A0E80E0F1F1F0A1E511D601B710B80098A
:106D1000B50B48F4600F711F801DB51F0E1B1F0BB4
:106D20000A0A510907C02E0F3F1F4A1F0E0F1F1FCF
:106D30000A1E511D660F771F881FBB1FA695F7956A
:106D4000E795F8F60617170708065B07211D311DA2
:106D5000411D0F911F91B901842F9158880F96956D
:106D6000879508959B01AC012CCFDF93D92FA3DE2B
:106D7000E695D7952AED3FE049E45FE3B33A620731
:106D8000730784079507D7952AF0A2EA49EC906823
:106D90008EDCC1DEE3EBF0E06EDEDD0F0BF00ADF30
:106DA000DD0F0BF49058DF910895882371F4772359
:106DB00021F09850872B762F07C0662311F499276E
:106DC0000DC09051862B70E060E02AF09A95660F16
:106DD000771F881FDAF7880F9695879597F908959A
:106DE0009F3F49F0915028F4869577956795B79520
:106DF0009F5F80389F4F880F9695879597F90895E4
:106E000091505040660F771F881FD2F70895AA1B34
:106E1000BB1B51E107C0AA1FBB1FA617B70710F085
:106E2000A61BB70B881F991F5A95A9F780959095B7
:106E3000BC01CD01089597FB092E07260AD077FDE6
:106E400004D0E5DF06D000201AF4709561957F4FDD
:106E50000895F6F7909581959F4F0895A1E21A2E17
:106E6000AA1BBB1BFD010DC0AA1FBB1FEE1FFF1FEE
:106E7000A217B307E407F50720F0A21BB30BE40B3E
:106E8000F50B661F771F881F991F1A9469F7609585
:106E90007095809590959B01AC01BD01CF0108953F
:106EA00097FB092E05260ED057FD04D0D7DF0AD058
:106EB000001C38F450954095309521953F4F4F4F29
:106EC0005F4F0895F6F790958095709561957F4F87
:106ED0008F4F9F4F0895EE0FFF1F0590F491E02D07
:066EE0000994F894FFCFB5
:106EE600256300256325630025632532692563250F
:106EF6003032697C25632532692563253032690085
:106F060025352E3066256300256325312E35662509
:106F160063002563253569256300256325352E32F3
:106F2600662563006D616E00737431007374320000
:106F360073743300737434007374350073743600DD
:106F460070682000636C200076722000686C200058
:106F560061702000727462006C616E0070702000B7
:106F6600706F69006163200000617420002563254D
:106F76007300256325332E30692563002534692582
:106F860063256300256325336925630025737C2506
:106F960063257325630020C0C0C0C0C0C7C0C0C081
:106FA600C0C0200025342E306625630025632533B6
:106FB6002E3066256300256325352E306625630051
:106FC60025632531312E36667C25632531312E36F3
:106FD600660025632532690025332E316625630058
:106FE6002020202020202020202020200020206477
:106FF600697361726D6564202000206E6F20746570
:107006006C20636F6D2000206E6F206770732066A2
:1070160069782000202062617474206C6F772020CC
:10702600006C696E6B207175616C697479006D61B5
:1070360067207761726E696E67006D6167206372A3
:1070460069746963616C00206D61672020657272E6
:107056006F72200025730020008A060000E803E80E
:1070660003E803E8039DFF016401000000007B05BF
:107076000C3379047C047F048204A12900070E09DD
:107086001C1B1215383F363124232A2D70777E7942
:107096006C6B6265484F464154535A5DE0E7EEE932
:1070A600FCFBF2F5D8DFD6D1C4C3CACD90979E9922
:1070B6008C8B8285A8AFA6A1B4B3BABDC7C0C9CE12
:1070C600DBDCD5D2FFF8F1F6E3E4EDEAB7B0B9BE02
:1070D600ABACA5A28F88818693949D9A2720292EF2
:1070E6003B3C35321F18111603040D0A5750595EE2
:1070F6004B4C45426F68616673747D7A898E8780D2
:1071060095929B9CB1B6BFB8ADAAA3A4F9FEF7F0C1
:10711600E5E2EBECC1C6CFC8DDDAD3D4696E6760B1
:1071260075727B7C51565F584D4A4344191E1710A1
:1071360005020B0C21262F283D3A33344E49404791
:1071460052555C5B7671787F6A6D64633E39303781
:1071560022252C2B0601080F1A1D1413AEA9A0A771
:10716600B2B5BCBB9691989F8A8D8483DED9D0D761
:10717600C2C5CCCBE6E1E8EFFAFDF4F3C2C0C0C16C
:10718600C0C0C1C0C0C4C0C0C1C0C0C1C0C0C3C0EF
:10719600C0C1C0C0C1C0C0C5C0C0C1C0C0C1C0C0E0
:1071A60000000000B72A0C33282A582A882AA52A64
:0871B6003E2AC6290C2B7C2B9C
:00000001FF
